:020000040000FA
:100000000C943F120C9467120C9467120C941027F6
:100010000C9467120C9467120C9467120C9467127C
:100020000C9467120C9467120C9467120C9467126C
:100030000C9467120C9467120C9467120C9467125C
:100040000C94C6260C9467120C9494260C946E267D
:100050000C9467120C94E7270C9467120C946712A7
:100060000C9467120C94671207634236B79BD8A7AB
:100070001A39685618AEBAAB558C1D3CB7CC5763CD
:10008000BD6DEDFD753EF6177231BF000000803F7B
:1000900005A84CCDB2D44EB93836A9020C50B9914E
:1000A0008688083CA6AAAA2ABE000000803F080055
:1000B0000000BE922449123EABAAAA2ABECDCCCCE7
:1000C0004C3E00000080BEABAAAAAA3E0000000081
:1000D000BF000000803F0000000000084178D3BB53
:1000E0004387D1133D190E3CC3BD4282AD2B3E6800
:1000F000EC8276BED98FE1A93E4C80EFFFBE01C4F1
:10010000FF7F3F0000000000800400003FF0383017
:1001100033103F90381033902790261030903FF0E6
:1001200000008004800400003FF03DF020103BF010
:100130003B7030302B502AD031B03FF000008004AB
:10014000800400003FF038703030231027902010DA
:100150002010279027903FF00000800480040000CA
:100160003FF03CF03CF020102490249020103CF014
:100170003CF03FF000008004800400003FF037B006
:1001800023103030387038703030231037B03FF0E3
:1001900000008004FCF4F860E044C08CC11CC22C58
:1001A000C44CC88CD10CA204C4048FFC187CBCFCC9
:1001B0008000BFF81FF8B0281FF8B4081FF8B10876
:1001C0001FF8B048BFF8B288BFF880008000BFF8C1
:1001D0001FF8B0081808B9E819B8B8381838B9B80D
:1001E000B9F8B0F8BFF8800015543FF815503FF04B
:1001F0001550387010203104138C22A817FC2AA83F
:100200000000000015543FFC15543FFC15543C04FD
:1002100014043CFC14543CFC005400A800000000F2
:10022000800400003FF03CF034B0249024902790EC
:100230002310303038703FF000008004FF7CFE7CDB
:10024000FCECE8DCC84C984C882408200000000036
:10025000000000008004E01CF3FCE7FCCE0C8E1CC8
:100260009F9C1F3C1F0C0E0C0FFC87F881E4C00CF8
:10027000E01CF87C000458085808580840087FF82B
:1002800060185FE85B685FE85B681CE85FE8000097
:10029000800400003FF03CF03CF03CF020102010C7
:1002A0003CF03CF03CF03FF000008004F87CF7BCF0
:1002B00000007FF80000BFF4AB54AB54AB54AB5418
:1002C000AB54AB54BFF4C00CF03CCE0CBF04B30431
:1002D00073007F007E007C007C007C60BC64BE04F8
:1002E000CF0CF03C81DC559C29045500299055D059
:1002F00003FCFF002E00267002508270E600EE0420
:10030000800C001C3FF43FE03FC4378C2318303092
:1003100038703CF03FF03FF000008004058074B876
:1003200057A876B80580F97C4694AAA8F97C068877
:1003300074A8578C75740698F03CCE4CBC34B81435
:10034000188010804230607860F844C08004B8841F
:10035000CFCCF03CE01CC00C8FC49FE49FE49FE432
:1003600000000300030003000780078003008004EF
:10037000F87CE01CC00CCFCCCFCCCFCCCFCCCFCC3A
:10038000CFCCCFCCC84CCFCCC00CE01CFCFCF87C54
:10039000E01CC00CC00CC00CC00CC00CC00C800415
:1003A0008004FFFCF87CFCFC8004000020001000AE
:1003B00008001000270000000000000000000000FE
:1003C00000008004C3FC18001800C3FCFFFCFF0CF5
:1003D00000600060FF0CFFFCF0FC06000600F0FC73
:1003E0008FC4102020104CC89FE43DF03DF01DE06C
:1003F0003EF03F709FE48CC400003030F87CF33C4A
:10040000F4BCF6BCF4BCF6BCF4BCE49CC84CD02CE8
:10041000D02CC84CE79CF03C882408203830383079
:10042000383038303830383039303BB03FF03FF07A
:1004300000008004F21415F0CADFB8CCF0D699E8B9
:10044000AEA4DFEEE8F21D1E08F21C08F21A1B082B
:10045000F0714601F046464A01F219F051F218F0E7
:100460005A8DF0C0DAEEAEF0C8B8A5F1302924F00C
:10047000B599E1A4BDF21415F0CBEEAEBDF218F0C3
:100480005A8DF21617F21415F0CBEEAEBDF2161718
:10049000F0BCCA9EE0BDF21415F21213F21011F274
:1004A0000C0DF094F20E0FF0A2D8DFCBE1EEACDC35
:1004B000E8F20AF08CF20BF04A8DF209F08DF09719
:1004C000C59BBDF20708F21F20F2040506F097DE77
:1004D000EED5F0CBABEEF0AEA4DFEEE8F0A8E8BDD1
:1004E000E2EEE0F0B499D3EEF200010203F0CCDFCB
:1004F000B0B8BD5361766500466C6970004D6169A6
:100500006E2053637265656E004A5000454E00438D
:100510004E00594553004E4F004F4E004F46460087
:10052000496E666F73004269670050494400446930
:1005300072656374005361766500426F6F73740077
:100540004F666600536C65657000536176650042C6
:100550006F6F737400536C656570004465666175F8
:100560006C740053617665004164640044656C6599
:1005700074650052656E616D650043616C696272FD
:10058000617465004368616E6765005265747572D9
:100590006E0041626F7574004C616E67004C6F6352
:1005A0006B004C4F5720566F6C0042757A7A65721B
:1005B0000053637265656E00436F6E74726F6C00FA
:1005C00054696D65720054656D7000546970000067
:1005D000000000000F1DC20800054442080003840B
:1005E0005FBF000FE44410000115451000054CC921
:1005F0007F8009244F900007C4C11000054D413F82
:1006000000055443810007C44D0200054441140015
:10061000055541080007C8810400000000000000E3
:100620000000000001083FFE001FFF8100000040A5
:1006300002000007FE0FF800040208080004020888
:10064000880007FE08880004020888000402088861
:100650000007FE0888000402094800040202300076
:1006600007FE040C00040218040000000000000053
:100670000000000007FE13FE000402084000040210
:10068000084000040201FC0004023884000402084F
:10069000840007FE0FFF000402080000040209FEA8
:1006A00000040209020004020B020004020D020011
:1006B00007FE09FE00040201020000000000000025
:1006C0000000000001100080001FFF80800001106A
:1006D0003FFF00004004080007FC04080004440435
:1006E0001000044402100004440220001FFF812077
:1006F00000004000C00000A001300001100208000E
:10070000060C0C07001803B00200000000000000F7
:1007100000000000004000800000400080000FFF4B
:100720003FFF000841040800084104080008410494
:10073000100008410210000FFF02200008410120B4
:1007400000004000C00000400130000040020800EE
:1007500000400C07000040300200000000000000D4
:10076000000000001FDF10200002120C20000224F5
:10077000042000047F8020000424B820000FA488F7
:10078000500014BF88500004A488500004A4884876
:100790000004BF88880004A48A880007A48C840011
:1007A0000444890700008186020000000000000068
:1007B000000000000FF00491000440025200047F8A
:1007C000905400045088FF0007D084810004510039
:1007D0008100044901FF0007CA028100044404812A
:1007E00000044A1CFF0007EA0481000C5104810048
:1007F0000061C4850000408082000000000000000D
:100800000000000007FF802000008407FF00008434
:10081000040100008404010000840401000FFFC7EC
:10082000FF0000840400000084040000008405FF31
:100830000000840501000104090100010409010010
:10084000020411FF00040401010000000000000088
:1008500000000000008204FF00004402010007FFC6
:100860009021000010102100001017FD0000101052
:1008700021000FFFD06100001010A10000281121FD
:100880000000281221000044142100008210A10061
:100890000301D045000C00900200000000000000A1
:1008A00000000000084410FE00042810920005FF1C
:1008B00022920000103C920000100892001CFE10D2
:1008C0009200041020FE0004103E920005FF80926A
:1008D00000041000920005100E92000610309200E5
:1008E000041000FE00001000820000000000000064
:1008F0000000000007DF8840000A24104000114279
:1009000010FE00040022820002FF3D020008010ADE
:10091000420009F9103200090920120009F93E02CB
:1009200000090900020009090E020009F93022003D
:100930000805001400080200080000000000000084
:10094000000000000FC3F1E0000FE3F1F8000C70AD
:10095000C19E000C30C186000C30C183000C30C138
:1009600083000C60C183000C60C183000FC0C18391
:10097000000FC0C186000C00C186000C00C19800A9
:100980000C03F1F8000C03F1E0000000000000008F
:100990000000000000200820000FFF09FC000020DC
:1009A00008000000203E880003FE08500002020BF1
:1009B000FE0003FE0C4000020218400003FE2BFE66
:1009C00000020208480003FE0888000202085000E6
:1009D00002022830001FFF91CC000000000000013F
:1009E00004047C0000880444000FFF3F4400002002
:1009F00004440000200C440000200E44001FFF951A
:100A000044000020144400005024440000500444DA
:100A100000008804450001040485000603850300E6
:100A200018010400000000000000000000000000A9
:100A300000000000047E21FC0004421104001F7E1F
:100A4000090400044221FC000542110400067E1145
:100A500004000C0005FC0015FF880000040813FECC
:100A6000000448325200044F12520004481252004F
:100A700014A8125200091F97FF0000000000000098
:100A80000000000002103DFC0002102504000410CC
:100A900025040005FFBDFC000C102520000C3825A6
:100AA0002000143825FE0004543D20000454251075
:100AB0000004922510000511A5090006113D45000E
:100AC0000410258300041001010000000000000054
:100AD000000000001FC8102000124A0C20001AC994
:100AE00004200017480020001FFFB820000208085B
:100AF00050001FC8085000020808500003C80848EA
:100B0000001E1408880001540A880015220C840075
:100B10001443890700008106020000000000000263
:100B2000FE01000002823FFF00048202000004FE7A
:100B30000200000C1004FC00141004080005FF8CD7
:100B400010000410141000043825FF0004340410B1
:100B50000004520410000491841000051004500099
:100B6000041004200000000000000000000000004D
:100B70000000000002030010001FDC3EFE00089091
:100B8000021200051004FF001FDF84120002120C85
:100B9000FE001FD2021000021222FE000A92141060
:100BA000000A5214100012220DFF00022208100049
:100BB0000A42141000040223FF000000000000009D
:100BC000000000000F78BC20000948A45000094A2A
:100BD000A85000094AA88800094AB104001FFEAACB
:100BE000FB00094AA42000094AA42000094AA7FEE4
:100BF00000094AB420000948A924000B48A2220099
:100C0000088AA4A200111920400000000000000082
:100C1000000000000020008000005001FC0000885F
:100C2000010400010403080006FB0490000800C052
:100C3000600007DF018000045106000004511BFE24
:100C400000045102020007D9020200045602020009
:100C5000001003FE0000100202000000000000006F
:100C6000000000000208209000027F9890001F8082
:100C700009FF00022201100006218B100007628D7F
:100C8000FE000AA20910000A14111000121431FE0D
:100C900000020811100002141110000222111000AD
:100CA000024391FF000281110000000000000000DB
:100CB00000000000100700000008F83FFE0004805C
:100CC000200200008020020000BE23E2001C8222DD
:100CD000220004A42222000494222200048822225A
:100CE00000049423E20005222002000542200200B5
:100CF0000A003FFE0011FFA00200000000000000FB
:100D00000000000000820FFE00004400400007FFCA
:100D10008040000010004000001000400000101F44
:100D2000FF800FFFC040000010004000002800407E
:100D30000000280040000044004000008200400005
:100D40000301C140000C0080800000000000000989
:100D5000FF00400004203FFF00042000000000FED0
:100D60000000001C420FFC00044200000007FF804E
:100D7000000004000FFC0004FF00000004810000DC
:100D80000005810FFC00068108040004FF08040030
:100D900000810FFC000000000000000000000000C7
:100DA0000000000000401F7E001FFF840200108032
:100DB0008442000A4A0442000A3108420012C50F68
:100DC00042000304197F001DF829010000400901B9
:100DD00000084209FD00084209010008420F010015
:100DE0000FFE0905000002000200000000000000E4
:100DF0000000000001000FFE00010008200003FFBA
:100E00000820000201082000042208200008200B0E
:100E1000FE00102008200000500828000050082480
:100E20000000880822000088102000010410200023
:100E30000203A7FF000C01000000000000000000FA
:100E40000000000000400080001FFF9FFC000040E9
:100E50000410000FFF02200000003FFF000FFE0003
:100E6000000008420FF80008420808000FFE0808BA
:100E70000008020FF8000800080800080008080031
:100E800008000FF800100008080000000000000033
:100E90000000000007FE0FF800040200000004023A
:100EA00000000007FE00000004023FFE00040200F4
:100EB000800007FE008000009004900008910C88DC
:100EC00000069310860002942082000090008000AB
:100ED00000900280001FFF81000000000000000061
:100EE00000000000041012020005FF9FD200050060
:100EF0009212001E28A2120004443FF20004820253
:100F0000120006000212000CFE1FD2001410125232
:100F10000004101242000410134200041012820058
:100F200015FF820A00080002040000000000000013
:100F300000000000002000000000203E04001FFF11
:100F4000A204001000A2FF0000012204000FFE22F4
:100F5000040000403E4400004022240004402224BB
:100F600000047C22040004402204000A403E0400E5
:100F7000094022240010FF80140000000008000037
:100F80000000000010FE08200008820BFF00048211
:100F90000A010010FE3C51000882088800088209FE
:100FA000040002FE0C0000040019FC0009FF2820C8
:100FB0000019290820000929082000092908200013
:100FC00009292BFF000BFF9000000000000000002B
:100FD000000000001F7F90F80001080888000A1038
:100FE000088800047F0107001FC13A000005490975
:100FF000FC000449088400044908880004490848A2
:1010000000044908500004490A200004160C580046
:10101000142189870008C086020000000000001F1C
:10102000E03FF07038601860186018FFFCFCFCFCB2
:10103000FCFCFCF87CF87CFCFC7FF81E1033382D9F
:101040007C25382D3825382D386D80DEC0BF40BF57
:1010500040DEC061803F007FF0FFE0C008C01CC0E0
:1010600038C870DCE4CFCCC78CC30CC00CC00CFFFC
:10107000FC7FF8000006000C0018F838F0303070E3
:1010800060707878F878003C023F0C1FF80FF0038E
:10109000C000007FF8FFFCC00CC30CCB4CDB6CDB4A
:1010A0006CD86CDCECCFCCC78CC00CFFFC7FF80399
:1010B0000007800FC00CC01CE01CE03CF03CF07F3F
:1010C000F87FF8FCFCFCFCFFFC7FF811408200215B
:1010D000208FE023FC82004A23E200FE209FF013D1
:1010E000F880802220C0804221BFF0FBFA88800275
:1010F000208480022084801A208080E3FE82800287
:101100000101000F421FC078411040084090400884
:10111000421FC008411040FFFD104008405FC0085A
:1011200040800008413FE008432520104125201061
:101130004125202041252040417FF07FF848800252
:101140000049000201FFF00201001002027F20228C
:1011500000410023F07F00220008002200FF8022CF
:101160000088802200888022008A8022008900FF77
:10117000FC080023F21FC022111040FBF090402217
:10118000121FC02A11104033F1104060005FC0AF41
:10119000FC800020413FE0224325202279252022A7
:1011A000412520A541252048FD7FF01083DFC01098
:1011B000825040208250402FFFDFC0608252006189
:1011C000C25200A1C25FE022A3D20022A251002499
:1011D000925100288E5090308BD45020825830206D
:1011E000801010104047C017FC44402003F44023F7
:1011F000F844406208C440A3F8E440200154402F62
:10120000FD44402806444023F844402040445020F8
:10121000404850214050302080400020921FC03D67
:10122000F990402090904040901FC07BFF0000A0AC
:10123000013FE021F90200FD09020021097FF021B0
:10124000F90500210945002909888031F91070212C
:1012500008202025004300202070F8754077557540
:101260007740403E4A5E2B5E4A6B627F352F357F6A
:101270007C5B5E247B0E3A047E017E4A5E69063A00
:101280002F3F6B7E46403F41497F494102626B6B75
:101290006B62026A6B147D577D10413F55553D5777
:1012A00051213F2D7F2A122E0A775A505A770A2051
:1012B00024137D5553707A2A7B021A437A4A525E70
:1012C0002B5E424A415F353F555F417D14577D0E8D
:1012D000407F7F1B54167D1654493A407E57567600
:1012E000423F427E7E427E047E51377D3750127AE5
:1012F0001752761E127F557F145D7F557F557F7F75
:10130000553D577F55377817457F7F2B7B287B2BA3
:101310007F1E12127F12121E7F416B7F6B517F5214
:101320005A573A575A52007F494949497F22122A4F
:101330007F2A1222166A5E735662160937315F15CC
:101340005F7500000000002F000300033F123F16EE
:101350003F1A120824323D2A020100003E41413E5C
:10136000000A070A083E084020000808080020007C
:101370001008041C2A1C243E20322A24222A141875
:10138000143E2E2A121C2A12023A06142A14242A67
:101390001C002400402400081422141414221408F1
:1013A00002290612291E3E093E3F251A1E21213F11
:1013B000211E3F25213F05011E21393F083F213FC6
:1013C0002110201F3F043B3F20203F063F3F013EAE
:1013D0001E211E3F09061E215E3F093622251901E6
:1013E0003F013F203F3F100F3F183F330C33033C7A
:1013F00003312D23007F41153E15417F000201027C
:1014000040404000010218243C3F241818242418AE
:10141000243F182C2C043F0548543C3F0438003D21
:1014200000403D003F0834013F003C1C383C04387C
:101430001824187C241818247C3C0804283C140424
:101440003E243C203C3C100C3C303C2418244C50A6
:101450003C24342C083641007F004136080101014C
:101460001028101F010120203E1020000008002538
:10147000150F241C0C103804180C3828382828188C
:101480003C083C18283820242C3C2C2C1C04080830
:10149000211D07083C0306231E223E22120A3F326A
:1014A0000F3E0A3F0A24130E271E0222223E271255
:1014B0000F2525102119273F222E21160F241B0E40
:1014C000251F0526261E251D053F0408241F042070
:1014D0002222251927123B1620100F3C013E1F2403
:1014E0002421110F0C031C1A3F1A091927222A2A3A
:1014F000382730320C13053F25023F0E213F2025AF
:10150000253F25251D07201F3C3F203F20103E2260
:101510003E23110F212118010001020502000000E5
:1015200000000000002040000000000000205020CB
:10153000000000000050300000000000006060006B
:101540000000000000000018180000000000003635
:1015500036000000000000563600000000000201C6
:1015600051090906000000005F00000000000000B3
:10157000007F41410041417F000000000000000069
:101580003F010101004040407E0000000000003F9C
:10159000213D05070070505E427E00000000000003
:1015A000007F63410041637F0000000000080808DD
:1015B0007F08080800080808080808080044444490
:1015C0005F444444004122140814224100080808E2
:1015D0002A080808001414141414141400143414E1
:1015E0001C141614000808141414222200222214B9
:1015F00014140808000205023C42422400002B2C6F
:10160000782C2B000000242A7A2F2A1200001C625A
:10161000322E23140020545E254142200042251220
:10162000082452210020623E633E230200205649D6
:1016300055225840000022147F142200001C225919
:10164000554D120C0000004A555529000004643C19
:10165000173C64040004643C1F3C6404001C2241E9
:101660004141221C001C3E7F7F7F3E1C001C225DEE
:10167000555D221C000814224122140800081C3E5B
:101680007F3E1C08007F41414141417F007F7F7FB9
:101690007F7F7F7F0040704C434C70400040707CE7
:1016A0007F7C704000010719611907010001071FC5
:1016B0007F1F07010049221449142249000505052E
:1016C0007D05050500080808082A1C0800081C2AD2
:1016D00008080808000004027F020400000010202F
:1016E0007F20100000003E414141413E0000004289
:1016F0007F400000000062515149494600002241EC
:10170000494949360000302824227F2000002F4517
:101710004545453900003E4949494932000001012B
:101720006119050300003649494949360000264938
:101730004949493E000020547E3414600020527F05
:101740002A1A4A3000003C4020041800001E2040A5
:10175000200204180000104A4A2A10000000084520
:10176000454525180000482A3A4A40000000442513
:10177000153D45400000247E145024000022527F75
:101780000A484A340044344F443804180044344F63
:101790004439041900002A5A4B4E5A0800002A5AAC
:1017A0004B4E5B080000081414224100000008148E
:1017B00014224504003F0004443F0404003F000499
:1017C000443F0405000020524242424000002052A3
:1017D000424342410000245444475C040000245426
:1017E00044475C050000003F404040200000003FAF
:1017F000404140210002020A563F02020002020A52
:10180000563F02030004043F44545F440004043F75
:1018100044545F45000008093D4B49080000080991
:101820003D4B490A00423A072254444400423A07D9
:1018300022554445000002124E4B4A32000002126B
:101840004E4B4A3300001010484830000004040298
:101850002222221C000404022223221D0000020274
:101860001A254341000002021A2543450000205773
:1018700048484444000020574849444500120A277C
:1018800052503A24007F00205242424000304E38ED
:10189000540F64780024147F0422523C0018241250
:1018A0004E422418007F002454543F44007F0024FB
:1018B00054543F45007F002454563D4600023A47A9
:1018C00040413E0400023A4740413E0500023A478B
:1018D00040433D06004030404D32106000403040F3
:1018E0004D321161004030404D3215620008040253
:1018F0000408101000080402040910110008040272
:10190000040A1512007F006A6A7E2A4A007F006A74
:101910006A7F2A4B007F006A6A7E2D4A00006A6A4D
:101920006A7F2A4A0030291D4B483C1000122A7F4A
:101930004240422400304E38540F443800000A3EE2
:101940004B4A4A300000080E384614080004071CB1
:1019500062030A0400001C483E241800001E0452C2
:101960003F12120C00002050503E48000000205052
:10197000503F244400001C51494A483000000F42A7
:1019800041211E00000010696D4B49300024147F76
:1019900004023E40000010494D4B49300000281819
:1019A0007E0844380024147F0442423C003049251C
:1019B0001F245438004028255735284000100A2E8F
:1019C0005B724A480040300C334040200000044421
:1019D0003C140C00000001413D09050300002020DB
:1019E0001078040000001010087C02010000184864
:1019F0004C281800000006424322120E0000404806
:101A000078484000002022223E2222200000282880
:101A1000587C0800002222124A7F02020000422263
:101A20001F02427E000042221F02427F000012126B
:101A30001F721210000012121F72131000000844CF
:101A40004322120E000008444322120F00080742EE
:101A5000221E020200080742221F02030000424227
:101A60004242427E000042424243427F0002024F15
:101A700042221F020002024F42231E030000454A79
:101A80004020100C0000454A4021100D0040422229
:101A9000221A264000404222221B26410004043F15
:101AA0004444544C0004043F4445544D0000014656
:101AB0004020100F000001464020110F0000084494
:101AC0004B2A120E000008444B2A120F00080A4A43
:101AD0003E09090800080A4A3E09080900001840A2
:101AE0005820180000020C424C20100E00020C423C
:101AF0004C21100D000405453D0505040004054575
:101B00003D0504050000007F080810000000007F6C
:101B100008091001000444241F04040400202222A8
:101B200022222220004041251519270000202212E0
:101B30007B06122000404020100807000040300EB5
:101B400000020C700040300E00020D710040300E9B
:101B500000020D7200003F484848444400003F48DE
:101B60004849444500003F48484A45460000024273
:101B70004222120E000002424223120F00000242D3
:101B80004222150E00080402040810200008040276
:101B90000409102100080402040A15220024144438
:101BA0007F041424002414447F05142500241444C5
:101BB0007F0615220002021222520A060000212589
:101BC000294A42000040704C4350204000404424C9
:101BD00014083700000008093F4949480000101C5C
:101BE000680818000004040F74020A060000404848
:101BF0004878400000202222223E2020000000449D
:101C000054547C000000424A4A4A4A7E000004457F
:101C10004525150C00000F4040201F000040201EED
:101C2000007F20100000007F4020100800007E424E
:101C30004242427E00000C4444241C000000064244
:101C40004222120E0010121E12127F1200202222B7
:101C50003A262220000001454525150F000041428B
:101C60004020100C000006424322120F00004828BA
:101C70001C4878000000100C4838080000080404D4
:101C800008101008000800000800000800040808F8
:101C900008080808000808080808080808060505D4
:101CA0000706040903030504090A080303030603DE
:101CB00005030305050306040405050405040403E0
:101CC00004090503CB05C605C005B805B105AA057D
:101CD000A2059D05980592058B0584057A05730577
:101CE0006C05680563055B0555054F054A05440508
:101CF00040053A0535052E052A05260520051C0553
:101D00001905160512050F050C050905FD04F80453
:101D1000F3043E0053656C656374205469700000E1
:101D2000000000003E5B4F5B3E3E6B4F6B3E1C3E37
:101D30007C3E1C183C7E3C181C577D571C1C5E7F4B
:101D40005E1C00183C1800FFE7C3E7FF00182418CA
:101D500000FFE7DBE7FF30483A060E2629792926FF
:101D6000407F050507407F05253F5A3CE73C5A7FE9
:101D70003E1C1C08081C1C3E7F14227F22145F5F3F
:101D8000005F5F06097F017F006689956A60606079
:101D9000606094A2FFA29408047E040810207E20B4
:101DA0001008082A1C08081C2A08081E1010101009
:101DB0000C1E0C1E0C30383E3830060E3E0E06004F
:101DC0000000000000005F00000007000700147F13
:101DD000147F14242A7F2A1223130864623649567A
:101DE00020500008070300001C2241000041221C73
:101DF000002A1C7F1C2A08083E080800807030005A
:101E00000808080808000060600020100804023E6E
:101E10005149453E00427F400072494949462141AF
:101E2000494D331814127F1027454545393C4A491E
:101E3000493141211109073649494936464949295D
:101E40001E0000140000004034000000081422416D
:101E50001414141414004122140802015909063EF6
:101E6000415D594E7C1211127C7F494949363E41F1
:101E70004141227F4141413E7F494949417F090912
:101E800009013E414151737F0808087F00417F41AD
:101E9000002040413F017F081422417F40404040E4
:101EA0007F021C027F7F0408107F3E4141413E7F3C
:101EB000090909063E4151215E7F09192946264933
:101EC00049493203017F01033F4040403F1F20400A
:101ED000201F3F4038403F63140814630304780414
:101EE000036159494D43007F4141410204081020DC
:101EF000004141417F040201020440404040400053
:101F00000307080020545478407F2844443838445C
:101F1000444428384444287F385454541800087ED8
:101F2000090218A4A49C787F0804047800447D402A
:101F3000002040403D007F1028440000417F4000C9
:101F40007C047804787C080404783844444438FCE1
:101F50001824241818242418FC7C08040408485465
:101F600054542404043F44243C4040207C1C204022
:101F7000201C3C4030403C44281028444C90909019
:101F80007C4464544C440008364100000077000053
:101F9000004136080002010204023C2623263C1EB2
:101FA000A1A161123A4040207A3854545559215524
:101FB0005579412154547841215554784020545545
:101FC00079400C1E52721239555555593954545492
:101FD0005939555454580000457C410002457D4212
:101FE0000001457C40F0292429F0F0282528F07CC8
:101FF000545545002054547C547C0A097F49324989
:102000004949323248484832324A4848303A4141D8
:10201000217A3A42402078009DA0A07D3944444472
:10202000393D4040403D3C24FF2424487E494366DE
:102030002B2FFC2F2BFF0929F620C0887E090320B7
:10204000545479410000447D413048484A32384078
:1020500040227A007A0A0A727D0D19317D262929DB
:102060002F28262929292630484D402038080808DD
:102070000808080808382F10C8ACBA2F102834FAFE
:1020800000007B000008142A142222142A14089548
:1020900000220095AA005500AAAA55AA55AA000038
:1020A00000FF00101010FF00141414FF001010FFA8
:1020B00000FF1010F010F0141414FC001414F700BA
:1020C000FF0000FF00FF1414F404FC141417101F89
:1020D00010101F101F1414141F00101010F0000017
:1020E00000001F101010101F10101010F010000032
:1020F00000FF101010101010101010FF1000000042
:10210000FF140000FF00FF00001F10170000FC0478
:10211000F414141710171414F404F40000FF00F75B
:1021200014141414141414F700F7141414171410BE
:10213000101F101F141414F4141010F010F00000ED
:102140001F101F0000001F14000000FC140000F00E
:1021500010F01010FF10FF141414FF141010101FB3
:1021600000000000F010FFFFFFFFFFF0F0F0F0F0C4
:10217000FFFFFF0000000000FFFF0F0F0F0F0F38E1
:10218000444438447C2A2A3E147E02020606027E1B
:10219000027E0263554941633844443C04407E203A
:1021A0001E2006027E020299A5E7A5991C2A492A4B
:1021B0001C4C7201724C304A4D4D303048784830DA
:1021C000BC625A463D3E494949007E0101017E2AD2
:1021D0002A2A2A2A44445F444440514A4440404405
:1021E0004A51400000FF0103E080FF000008086B37
:1021F0006B083612362436060F090F060000181831
:102200000000001010003040FF0101001F01011EFE
:1022100000191D1712003C3C3C3C0000000000006F
:10222000000000240027002A0000000000250028EC
:10223000002B0000000000230026002900040404F5
:10224000040404040402020202020203030303035F
:10225000030102040810204080010204081020013C
:10226000020408102000000008000201000003041E
:10227000070000000000000000AED5F0A83FD3002A
:10228000408D14A1C8DA1281CFD9F1DB40A4A6AFEA
:10229000200021007F220007506C65617365207764
:1022A000616974004144433A200074656D703A20BE
:1022B00000536574206D65617375726564005374B5
:1022C00065703A2000FFFFFFFFFFFF8003867080EC
:1022D000038003867080039FF3E1309FF39FF3E157
:1022E000309FF3983301CC9833983301CC983398CE
:1022F0003387C098339833E1C098339833E1C0985E
:10230000339FF398C09FF39FF398C09FF3800366B9
:10231000CC8003800366CC8003FFFF010CFFFFFF2E
:10232000FF01001FFF810061301F3F873CE6FC87F3
:1023300033873CE6FC87F3F8039E0F1F03F8039EE8
:102340000F1F03E13CFE0C07CFE13CFE0C07CF99C9
:10235000033E3086C3E6CF380F9EF3E6CF380F9E9C
:10236000F39E0327CC81039E0327CC8103E0FFE18A
:102370000CE6CFE0FFE10CE6CF9803060000FF98E3
:1023800003060000FFFFFF1EF0F80380036630998C
:10239000C38003663099C39FF3010CF8FF9FF301DC
:1023A0000CF8FF9833393C01CF9833393C01CF9872
:1023B00033FF0C793F98333ECCE0F398333ECCE0CA
:1023C000F39FF33E0098CF9FF33E0098CF80033EEB
:1023D00030E7C380033E30E7C3FFFFFFFFFFFFFF8F
:1023E000FFFFFFFFFF3030300076312E372B0056D5
:1023F00000560043000FE01FC01FC03F803FF87F22
:10240000F07FE007C007800F000E001C00180010CE
:102410000014A03FF07FF8E01C6E18EC1C681860F8
:1024200018E01C6058E01C7FF83FF014A0455252A1
:102430004F5200484F4C44004845415400574F52BA
:102440004B5900424F4F535400534C454550004F99
:1024500046460000003BEC7BEE63E663E663E66322
:10246000E663E663E663666226600660067FFE3F1B
:10247000FC0000010204081020408000E82711241D
:102480001FBECFEFD8E0DEBFCDBF12E0A0E0B1E0CD
:10249000ECEFFFE602C005900D92AE3CB107D9F714
:1024A00027E0AEECB2E001C01D92A33EB207E1F717
:1024B00012E1CFE3D2E104C02197FE010E94DD3793
:1024C000CE33D107C9F70E942D280C94FC370C9409
:1024D000000080389105B0F46034710598F4E3E7AA
:1024E000F4E290E1969FD001A0781124A80F6770C4
:1024F000E60FF11D9491AE5CBC4F442321F08C910A
:10250000982B9C93089590958C919823FACFDF9205
:10251000EF92FF920F931F93CF93DF937C01D22E04
:102520008B01040F111DEB0177FF02C0D0E0C0E06A
:10253000C8010134110514F080E490E0C817D907F0
:102540003CF44D2DBE01C7010E9469122196F0CFC7
:10255000DF91CF911F910F91FF90EF90DF90089541
:10256000CF92DF92EF92FF920F931F93CF93DF935F
:102570006B01122FEC017C01E40EF11CCE15DF057E
:1025800044F4202F412FB601CE010E9487122196DC
:10259000F5CFDF91CF911F910F91FF90EF90DF90DA
:1025A000CF9008952F923F924F925F926F927F92B9
:1025B0008F929F92AF92BF92CF92DF92EF92FF9253
:1025C0000F931F93CF93DF9300D01F92CDB7DEB749
:1025D000C22ED12C9601280F391F37FD4FC08038ED
:1025E00091050CF04BC0E9824A017B013C01402E71
:1025F000512C160127E0220E311C93E035942794CC
:102600009A95E1F78B01B12CA12C1B821A82EA81E9
:10261000FB8183E0F595E7958A95E1F7EA0DFB1DCF
:10262000E80DF91DE4918A819B818770992720E844
:1026300030E002C0359527958A95E2F7C901F0E0B0
:10264000E223F923EF2B41F04981B8018A819B8174
:10265000860D971D0E9469128A819B8101969B833A
:102660008A838C159D059CF2A20CB31C0F5F1F4F33
:10267000C8018E199F09841595053CF20F900F90A3
:102680000F90DF91CF911F910F91FF90EF90DF900E
:10269000CF90BF90AF909F908F907F906F905F9002
:1026A0004F903F902F9008950F931F93CF93DF93F8
:1026B000EC018B0140E001960E94691240E0B801F4
:1026C000CE0101970E946912B8016F5F7F4F40E011
:1026D000CE010E946912B8016150710940E0CE013B
:1026E0000E94691240E0B801CE01DF91CF911F91A5
:1026F0000F910C94691280E0E2E3F3E081118FEF17
:10270000002481938193819381930394D1F7EFEC1B
:10271000F7E0178616861586148608956F927F92C5
:102720008F929F92AF92BF92CF92DF92EF92FF92E1
:102730000F931F93CF93DF93803891050CF057C010
:10274000603471050CF053C07B0137E0E322FF24B5
:1027500033E0759567953A95E1F7DB01B695BA2FA9
:10276000AA27B795A7955D01C0E8AC0EB11CA80ECD
:10277000B91EA80FB91FAE5CBC4F00E810E0081BE3
:10278000190B90E080E0E8E0F0E04F018E189F0820
:1027900030E0FA01E80FF91FC4917D906D01D1E09E
:1027A000CD1AD1080E2C01C0CC0F0A94EAF77C2A6E
:1027B000E6017882E114F10499F06730710581F047
:1027C000E491EC01CA0DDB1DCE5CDC4FF0E0082C7F
:1027D00002C0F595E7950A94E2F7F881EF2BE883BC
:1027E0000196821793071CF40817190791F6DF91D9
:1027F000CF911F910F91FF90EF90DF90CF90BF90FE
:10280000AF909F908F907F906F900895AF92BF92FE
:10281000CF92DF92EF92FF920F931F93CF93DF93AC
:102820006C017B018B01040F151FEB015E01AE18DB
:10283000BF08C017D10759F06991D601ED91FC91FD
:102840000190F081E02DC6010995892B79F7C5012A
:10285000DF91CF911F910F91FF90EF90DF90CF907C
:10286000BF90AF900895FC01538D448D252F30E02B
:10287000842F90E0821B930B541710F0CF9608958D
:1028800001970895FC01918D828D981761F0A28DBA
:10289000AE0FBF2FB11D5D968C91928D9F5F9F7380
:1028A000928F90E008958FEF9FEF0895FC01918D36
:1028B000828D981731F0828DE80FF11D858D90E0A3
:1028C00008958FEF9FEF0895FC01918D228D892F40
:1028D00090E0805C9F4F821B91098F739927089528
:1028E00082E397E00E94641421E0892B09F420E040
:1028F000822F089580E090E0892B29F00E947014C7
:1029000081110C9400000895FC01A48DA80FB92F2B
:10291000B11DA35ABF4F2C91848D90E001968F7307
:102920009927848FA689B7892C93A089B1898C9126
:10293000837080648C93938D848D981306C0028875
:10294000F389E02D80818F7D80830895EF92FF923F
:102950000F931F93CF93DF93EC0181E0888F9B8DC2
:102960008C8D98131AC0E889F989808185FF15C07C
:102970009FB7F894EE89FF896083E889F98980819F
:102980008370806480839FBF81E090E0DF91CF916E
:102990001F910F91FF90EF900895F62E0B8D10E090
:1029A0000F5F1F4F0F731127E02E8C8D8E110CC0FF
:1029B0000FB607FCFACFE889F989808185FFF5CF4A
:1029C000CE010E948414F1CFEB8DEC0FFD2FF11D91
:1029D000E35AFF4FF0829FB7F8940B8FEA89FB8987
:1029E00080818062CFCFCF93DF93EC01888D8823E5
:1029F000B9F0AA89BB89E889F9898C9185FD03C062
:102A0000808186FD0DC00FB607FCF7CF8C9185FF46
:102A1000F2CF808185FFEDCFCE010E948414E9CFF3
:102A2000DF91CF910895833081F028F4813099F0BF
:102A30008230A9F008958730A9F08830C9F0843039
:102A4000B1F4809180008F7D03C0809180008F77EA
:102A500080938000089584B58F7784BD089584B5F0
:102A60008F7DFBCF8091B0008F778093B000089569
:102A70008091B0008F7DF9CFCF93DF93282F30E086
:102A8000F901EB59FD4D8491F901EF5AFD4DD491B7
:102A9000F901E35CFD4DC491CC23A1F081110E94AA
:102AA0001315EC2FF0E0EE0FFF1FED5CFD4DA5912F
:102AB000B491EC91ED2381E090E009F480E0DF91A6
:102AC000CF91089580E090E0FACF1F93CF93DF93EA
:102AD000282F30E0F901EB59FD4D8491F901EF5AAF
:102AE000FD4DD491F901E35CFD4DC491CC23A9F0D7
:102AF000162F81110E941315EC2FF0E0EE0FFF1F2F
:102B0000E75DFD4DA591B4918FB7F894EC9111114B
:102B100008C0D095DE23DC938FBFDF91CF911F914A
:102B20000895DE2BF8CFCF93DF9390E0FC01EF5AAE
:102B3000FD4D2491835C9D4DFC0184918823C9F057
:102B400090E0880F991FFC01E15EFD4DA591B491C5
:102B5000FC01E75DFD4DC591D49161110DC09FB79A
:102B6000F8948C91209582238C9388812823288344
:102B70009FBFDF91CF910895623051F49FB7F894D1
:102B80003C91822F809583238C93E8812E2BEFCF6D
:102B90008FB7F894EC912E2B2C938FBFEACF1F9315
:102BA000CF93DF93182FEB0161E00E9493152097DC
:102BB00039F460E0812FDF91CF911F910C9465155E
:102BC000CF3FD10511F461E0F5CFE12FF0E0EB59F3
:102BD000FD4DE491E33031F140F4E130B1F0E23009
:102BE000E1F0C038D1057CF7E4CFE73029F1E830D7
:102BF00059F1E430B1F780918000806280938000C9
:102C0000D0938B00C0938A0004C084B5806884BDD3
:102C1000C7BDDF91CF911F91089584B5806284BDB7
:102C2000C8BDF7CF80918000806880938000D093EA
:102C30008900C0938800EDCF8091B00080688093B8
:102C4000B000C093B300E5CF8091B0008062809364
:102C5000B000C093B400DDCF3FB7F8948091F2028A
:102C60009091F302A091F402B091F50226B5A89BD1
:102C700005C02F3F19F00196A11DB11D3FBFBA2F0E
:102C8000A92F982F8827BC01CD01620F711D811DCE
:102C9000911D42E0660F771F881F991F4A95D1F753
:102CA00008958F929F92AF92BF92CF92DF92EF9250
:102CB000FF924B015C010E942C166B017C010E946B
:102CC0002C166C197D098E099F09683E7340810599
:102CD0009105A8F321E0821A9108A108B10888EEB5
:102CE000C80E83E0D81EE11CF11C81149104A104DC
:102CF000B10429F7FF90EF90DF90CF90BF90AF9095
:102D00009F908F9008952FB7F8946091EE02709184
:102D1000EF028091F0029091F1022FBF089584E9B3
:102D20008093BC008091BC0084FDFCCF089580930B
:102D3000BB0084E88093BC008091BC0087FFFCCF7F
:102D4000089584EA8093BC008091BC0087FFFCCF8B
:102D500088E70C9497160E94A11680E48093BB002C
:102D600084E88093BC00E2E3F3E09091BC0097FF1D
:102D7000FCCF91919093BB008093BC0097E0E2332D
:102D8000F90799F78091BC0087FFFCCF0C948F1650
:102D9000CF93C82F0E94A11680E00E9497168C2F17
:102DA0000E949716CF910C948F16480F592F511DE2
:102DB0004138510514F040E850E0481BFB0177FD15
:102DC000379633E0F595E7953A95E1F7F695FE2FBE
:102DD000EE27F795E795E80FF91FEE5CFC4F67705B
:102DE000772781E090E001C0880F6A95EAF7382FD5
:102DF000213041F4415078F08191DF011197832B0C
:102E00008C93F8CF8095415030F09191DF0111976C
:102E100098239C93F8CF0895CF92DF92EF92FF9280
:102E20000F93CF93DF936C017B01C42FD22F202F00
:102E30000E94D516B7016D0F711D61507109603484
:102E400071052CF4202F4C2FC6010E94D516202F7F
:102E50004D2FB701C6010E948712C6018C0F911D2C
:102E6000202F4D2FB7010197DF91CF910F91FF9048
:102E7000EF90DF90CF900C9487122F923F924F9259
:102E80005F926F927F928F929F92AF92BF92CF92FA
:102E9000DF92EF92FF920F931F93CF93DF93CDB703
:102EA000DEB72A970FB6F894DEBF0FBECDBF9A8368
:102EB00089836A3061F5DC0152968C91B8E08B9F72
:102EC00090011124E981FA8186859785820F931FED
:102ED000978786871586148681E090E02A960FB63C
:102EE000F894DEBF0FBECDBFDF91CF911F910F9140
:102EF000FF90EF90DF90CF90BF90AF909F908F901A
:102F00007F906F905F904F903F902F9008956D301D
:102F100019F329813A813A872987D9011C96AD9006
:102F2000BC90B0E8AB16B1040CF07BC0F901C684CC
:102F3000D784F0E4CF16D1040CF073C0D9015296B7
:102F40006C90529745E09501649E200D311D11242F
:102F5000121613060CF065C0262C312C910153E09B
:102F6000220F331F5A95E1F72C0D3D1D1216130643
:102F70000CF057C05196BC91BB83E985FA85F08966
:102F8000FC83649FB00111249B01215E324E3A8381
:102F90002983712CE981FA818491F5E07F1201C0C7
:102FA00080E0460138E0532E282F30E03E832D8309
:102FB0004C8080FF4B80411004C03B818C813817CE
:102FC000E1F010E000E00615C0F4D501A00FB11F3C
:102FD000B887AF83F12CE12CE61460F4B701680DDB
:102FE000791D442D8F8198850E946912BFEFEB1ADD
:102FF000FB0AF2CF0F5F1F4FE6CF8D819E81959523
:1030000087955A94820C931C5110CECF7394E9810A
:10301000FA813196FA83E983A20CB31CF6E07F12A1
:10302000B9CFA985BA8552962C915297422F50E07C
:103030001C968D919C91B6E02B9F800D911D1124C3
:10304000E985FA85958784872389222309F444CF6B
:103050006AEF64039001659F300D112420583F4FA3
:10306000281739070CF038CFDF010190F081E02DEF
:103070000190F081E02D6AE0CD0109952DCF0F93ED
:103080001F93CF93DF938C01D0E0C0E0F801EC0FE9
:10309000FD1F6491662341F08FEC97E00E943D177D
:1030A000892B11F02196F2CFCE01DF91CF911F91A4
:1030B0000F910895682F8FEC97E00C943D170895B9
:1030C00090E080E0089580917A00806980937A0092
:1030D0008EE480937C0061E070E080E090E00E94EC
:1030E000511683B7817F826083BF80E130E020E0AA
:1030F00093B7916093BF889593B79E7F93BF90914C
:103100007A0096FDFCCF4091780050917900240F11
:10311000351F815069F780917A008F7780937A000C
:1031200084E0369527958A95E1F750E040E064EB1E
:103130007BE281E190E00E945734C90108958091BB
:103140007A00806980937A0088EC80937C006AE042
:1031500070E080E090E00E94511683B7817F82602A
:1031600083BF80E270E060E093B7916093BF889581
:1031700093B79E7F93BF90917A0096FDFCCF2091EC
:10318000780030917900620F731F815069F7809148
:103190007A008F7780937A00769567957695679514
:1031A00062527A4090E080E00E94223326EF38E2BB
:1031B0004CE151E40E942735089590917A0090697E
:1031C00090937A008E50806480937C0083B7817FD7
:1031D000826083BF20E290E080E033B7316033BF8C
:1031E000889533B73E7F33BF30917A0036FDFCCFF0
:1031F0004091780050917900840F951F215069F714
:1032000020917A002F7720937A0025E09695879574
:103210002A95E1F708958FE00E94DD18A091F90248
:10322000B091FA029C010E94AB340E94243328E53D
:1032300039E743E353E40E9427350E94A035CB01D0
:10324000089580910203882369F086E00E943C156E
:10325000892B41F06AE070E080E090E00E94511616
:103260001092020308956F927F928F929F92AF9275
:10327000BF92CF92DF92EF92FF920F93CF93DF93A3
:103280007C01C62F01E020E340E370E060E00E9493
:10329000B012570123E0A20EB11C00E02AE24AE27C
:1032A00063E070E0C5010E94B01270E060E0C70109
:1032B0000E94541367013FE2C30ED11C70E060E02E
:1032C000C6010E9454136FE270E0C7010E945413BC
:1032D0006FE270E0C6010E945413EC2FF0E0EE0F95
:1032E000FF1FE556FE4F8080918053E0E52EF12CC4
:1032F000D12CC12C60E8662E712CD0E0C0E0FE011C
:1033000033E0F595E7953A95E1F7EC0DFD1DE80DF5
:10331000F91DE491CE0187709927930102C035957C
:1033200027958A95E2F7C901F0E0E223F923EF2B14
:1033300069F0CE01880F991F8C0F9D1F01E023E0DB
:1033400043E0B7018A0D9B1D0E94B0122196CE303A
:10335000D105A9F632E0C30ED11C83E0E80EF11CC2
:103360002DE2E216F10449F6DF91CF910F91FF9023
:10337000EF90DF90CF90BF90AF909F908F907F9015
:103380006F9008950F931F93CF93809159018823D5
:1033900099F0CFEF0FEE11E061E085E00E94651536
:1033A000C8010197F1F760E085E00E946515C8014A
:1033B0000197F1F7C15081F7CF911F910F910895B7
:1033C0002F923F924F925F926F927F928F929F9235
:1033D000AF92BF92CF92DF92EF92FF920F931F9323
:1033E000CF93DF9310E000E0D0E0C0E03EE3E32EB7
:1033F000F12C40ECC42ED12CAA24A394B12C60E271
:10340000662E712C70E4272E312C4C2E86E00E9403
:103410003C1521E0892B09F020E020930203F09273
:103420003103E0923003D0922F03C0922E03B0926A
:103430002D03A0922C0382E890E090932B038093BD
:103440002A0380912A0390912B0395958795582EF6
:103450009FE1591243C0F0923103E0923003D092C1
:103460002F03C0922E03B0922D03A0922C03EEEBFB
:10347000F0E0F0932B03E0932A039FE5592E0E947E
:103480007B1382E08093E1071093DC070093DB0756
:10349000E0E3F0E0F093DE07E093DD078EE50E94C5
:1034A0005A181092DC071092DB077092DE076092C8
:1034B000DD07912C812C841438F580912003F401D0
:1034C00096E0989FE00DF11D1124E55AFE4F808192
:1034D0000E945A18EFEF8E1A9E0AEDCFF0E65F12A7
:1034E000CECFF0923103E0923003D0922F03C092FE
:1034F0002E03B0922D03A0922C0330922B03209226
:103500002A0380E2582EBBCF1093DC070093DB0721
:103510007092DE076092DD07852D0E945A180E9486
:1035200021190E94AB1686E00E943C15892B09F0F8
:1035300088CF80910203811184CF80902003F6E030
:103540008F9E40011124C401855A9E4F4C01FC01FD
:10355000EC0FFD1F50820E94C2196AE070E080E00B
:1035600090E00E9451162196005F1F4FC530D10593
:1035700009F04BCFF4011582852DDF91CF911F917A
:103580000F91FF90EF90DF90CF90BF90AF909F9002
:103590008F907F906F905F904F903F902F90089505
:1035A0002F923F924F925F926F927F928F929F9253
:1035B000AF92BF92CF92DF92EF92FF920F931F9341
:1035C000CF93DF93CDB7DEB76E970FB6F894DEBF1B
:1035D0000FBECDBF80912703882309F4A7C11092A5
:1035E000D5021092D6021092D7021092D802809083
:1035F000D5029090D602A090D702B090D802409009
:103600001403509015036090160370901703A301E4
:103610009201C501B4010E94BA346B017C0120E023
:1036200030E0A9010E94CF3518160CF0A2C1C701E5
:10363000B6010E94A0351B017093D4026093D3029F
:1036400080915401882309F498C1609121037091FD
:10365000220380912303909124030E9499356E8B5D
:103660007F8B888F998FB10190E080E00E94223398
:10367000162F7E8F8D8F092FA090D102B090D2028D
:1036800080910A0190910B01A0910C01B0910D0164
:103690008D839E83AF83B887809106019091070147
:1036A000A0910801B091090189879A87AB87BC87EF
:1036B0008091020190910301A0910401B091050154
:1036C0008D879E87AF87B88B70E060E0211431044E
:1036D00009F47BC0B1016A197B0990E080E00E9487
:1036E00022336A8B7B8B8C8B9D8B6091CF02709188
:1036F000D002C501880F991F681B790B620D731DDD
:1037000090E080E00E94223369837A838B839C83DC
:1037100029853A854B855C855F776D817E818F81B8
:1037200098859F770E94BB342D853E854F855889AB
:103730005F770E94BB346B017C01AC019B016D8102
:103740007E818F8198850E942735212F3E8D4D8D5A
:10375000502F0E9483332B013C01A70196016985FC
:103760007A858B859C850E9427352A893B894C89DF
:103770005D890E9483339B01AC01C301B2010E94A9
:10378000BB342B013C01A70196016D857E858F8599
:1037900098890E94273529813A814B815C810E945A
:1037A00083339B01AC01C301B2010E94BB3423E30C
:1037B00033E343E550E40E9483330E949935198B2B
:1037C0009E8D9A8FAD8DAB8F0C8F8E899F89680FE0
:1037D000791F77FF02C070E060E0611592E0790721
:1037E00014F06FEF71E0072E000C880B990B0E940C
:1037F00024336B017C01C0922103D0922203E0921A
:103800002303F092240323E333E343E750E4612FDF
:103810007E8D8D8D902F0E948333A70196010E948B
:10382000833329893A8D4B8D5C8D0E9483332D81A2
:103830003E814F8158850E94BB3460930A0170938A
:103840000B0180930C0190930D012AE939E949E1BC
:103850005FE3612F7E8D8D8D902F0E948333A701B2
:1038600096010E9483332A893B894C895D890E9495
:10387000833329853A854B855C850E94BB346093F0
:1038800006017093070180930801909309012AE9CA
:1038900039E949E95EE3612F7E8D8D8D902F0E947D
:1038A0008333A70196010E94833329813A814B819A
:1038B0005C810E9483332D853E854F8558890E9407
:1038C000BB346093020170930301809304019093D1
:1038D0000501B092D002A092CF023092D202209283
:1038E000D102609121037091220380912303909172
:1038F00024030E94993589E06E960FB6F894DEBFD6
:103900000FBECDBFDF91CF911F910F91FF90EF9030
:10391000DF90CF90BF90AF909F908F907F906F90EF
:103920005F904F903F902F900C94CF15809126037D
:10393000609150017091510181110EC0809112036C
:103940009091130320912503BC01222329F060915B
:103950004F01680F792F711D90E080E00E942233A3
:103960006093D5027093D6028093D7029093D802C9
:103970003ECEC701B60190585CCE20E030E040E07A
:103980005FE3C301B2010E94BB349B01AC01C501DE
:10399000B4010E94CF3518164CF4109221031092F6
:1039A000220310922303109224039BCF80E090E027
:1039B000AFE7B3E48093210390932203A093230302
:1039C000B09324038ECF4F925F926F927F928F922B
:1039D0009F92AF92BF92CF92DF92EF92FF92CF93DE
:1039E000DF938090FB029090FC02A090FD02B090CB
:1039F000FE02C0912003D0E0C501B4010E949935B8
:103A00006B017C0120E030E048E453E4C501B401DF
:103A10000E941D3393E0CC0FDD1F9A95E1F7C25F42
:103A2000DE4F87FF31C02881398150E040E02551C9
:103A3000310941095109C701B6010E94B93728EC83
:103A400030E040E050E00E945734CA01B9016B5E9B
:103A50007F4F8F4F9F4F0E942433609314037093C6
:103A600015038093160390931703DF91CF91FF9076
:103A7000EF90DF90CF90BF90AF909F908F907F900E
:103A80006F905F904F9008954A805B80712C612CFD
:103A900020E030E04CE853E4C501B4010E941D333E
:103AA00087FF1FC088809980B12CA12CA7019601A7
:103AB000285C310941095109C301B201681979092A
:103AC0008A099B090E94B93720E530E040E050E0C8
:103AD0000E945734CA01B901680D791D8A1D9B1DCA
:103AE000BACF2C813D8150E040E0241935094609C8
:103AF0005709C701B60168517140810991090E94B7
:103B0000B93720E530E040E050E00E945734CA0168
:103B1000B901640D751D861D971D9DCFFC01019097
:103B20000020E9F73197AF01481B590BBC018FEC1E
:103B300097E00C9406148F929F92AF92BF920F93CE
:103B40001F93CF93DF93CDB7DEB7A1970FB6F8944D
:103B5000DEBF0FBECDBF19A2423008F44AE08E018D
:103B60000F5D1F4F842E912CB12CA12CA501940127
:103B70000E948934E62FB901CA01EA30F4F4E05D0D
:103B8000D801EE938D01232B242B252B79F790E080
:103B900080E0109719F0CD010E948E1DA1960FB6FE
:103BA000F894DEBF0FBECDBFDF91CF911F910F9173
:103BB000BF90AF909F908F900895E95CE1CF6F9296
:103BC0007F928F929F92AF92BF92CF92DF92EF92AD
:103BD000FF920F931F93CF93DF93B090200377242E
:103BE0007394B11001C0712C80914E018150990BDA
:103BF0001092310310923003880F991F90932F0376
:103C000080932E0381E090E090932D0380932C030A
:103C10008B2D90E0880F991F90932B0380932A039C
:103C200086E00E943C1521E0892B09F020E02093DA
:103C30000203FF24F39472E0972EE6E08E2EFCE060
:103C4000CF2ED12C0E947B13C0912A03D0912B033D
:103C5000D595C795EC2E8E011127C801870D911DB2
:103C600077FC9A958B199109712C97FD06C08330CA
:103C7000910514F082E090E0782EF092E007109227
:103C8000DF079092E1071092DC071092DB07109299
:103C9000DE071092DD0784E19DE10E943F1810923B
:103CA000E007F092DF071092DC071092DB07A72CE9
:103CB000072C000CBB08C501019654E0880F991F22
:103CC0005A95E1F79093DE078093DD0782E19DE14D
:103CD0000E943F186C2E671890E080E098012A1926
:103CE0003B09590120914E018C010F5F1F4F621655
:103CF000D0F4D092DC07C092DB07980144E0220F99
:103D0000331F4A95E1F73093DE072093DD078A0DD4
:103D10009B1D889E9001899E300D1124C901855AF2
:103D20009E4F0E948E1DC801639403301105D1F689
:103D30000E9421190E94AB1686E00E943C15892B37
:103D4000B9F480910203811113C00E94C219E0925C
:103D50002003DF91CF911F910F91FF90EF90DF90A3
:103D6000CF90BF90AF909F908F907F906F9008956D
:103D7000BC2E68CFCF92DF92EF92FF92CF93DF936A
:103D800097FF19C06B017C018DE20E945A18EC016B
:103D900066277727CB016C197D098E099F094AE0B8
:103DA0000E949B1D8C0F9D1FDF91CF91FF90EF9084
:103DB000DF90CF9008954AE0DF91CF91FF90EF9090
:103DC000DF90CF900C949B1D4F925F926F927F92E9
:103DD0008F929F92AF92BF92CF92DF92EF92FF921B
:103DE0000F931F93CF936B017C01742EAC019B0149
:103DF0000E942C36882399F08FEB92E0CF911F918F
:103E00000F91FF90EF90DF90CF90BF90AF909F9079
:103E10008F907F906F905F904F900C948E1D460115
:103E20005701E894B7F82FEF3FEF4FE75FE7C50181
:103E3000B4010E942C3681110DC02FEF3FEF4FE7E8
:103E40005FE7C501B4010E941D3318161CF483EC12
:103E500092E0D4CF2FEF3FEF4FE75FE4C701B60109
:103E60000E94CF3518161CF487EC92E0C7CF2FEFD5
:103E70003FEF4FE75FECC701B6010E941D3387FD9E
:103E8000F3CF20E030E0A901C701B6010E941D3345
:103E900010E000E087FF08C08DE20E945A188C01F4
:103EA000F7FAF094F7F8F094C0E060E070E080E09A
:103EB0009FE37C1641F020E030E040E251E40E94B4
:103EC0002735CF5FF6CFA70196010E94BB342B01A7
:103ED0003C010E94A0354B015C014AE00E949B1D01
:103EE0007C01E00EF11ECC23B1F1C501B4010E94AA
:103EF00022339B01AC01C301B2010E94BA344B01D1
:103F00005C018EE20E945A18E80EF91EC15018F1A9
:103F100020E030E040E251E4C501B4010E94833367
:103F20002B013C010E94A0354B01B12CA12C4AE091
:103F3000C501B4010E949B1DE80EF91EC501B40124
:103F40000E9422339B01AC01C301B2010E94BA342A
:103F50004B015C01DBCFC701CF911F910F91FF9007
:103F6000EF90DF90CF90BF90AF909F908F907F9019
:103F70006F905F904F9008954F925F926F927F92F3
:103F80008F929F92AF92BF92CF92DF92EF92FF9269
:103F90000F931F93CF93DF93C82F81E0DC2FD82797
:103FA000D093E007C093DF078093E1070C2F2EE04A
:103FB00046E661E370E081E090E00E940C172091FA
:103FC000280330912903253F81E03807B8F4A4E69F
:103FD000B0E00E94AB3424EF31E040E050E00E94BA
:103FE0005734BA01A9014E5F5F4F6F4F7F4F2EE0EC
:103FF00061E370E081E090E00E94B0128090D50211
:104000009090D602A090D702B090D802C501B4011A
:104010000E9499359B01AC01A4E6B0E00E94763481
:1040200024EF31E040E050E00E94573429013A018A
:1040300082E0480E511C611C711CC20102970C2FBA
:104040002DE043E062E370E00E94B012620183E081
:10405000C81AD10824E045E06CE370E0C6010E9474
:10406000B01281E0481A510831E3E32EF12C4D2FB4
:10407000B701C2010E9469128FEFE81AF80A8DE3B6
:10408000E816F104A1F7ED2E04E025E047E552E142
:104090006BE370E0C6010E94D2120C2F2EE047E1C4
:1040A00061E370E088E690E00E940C1760912103C4
:1040B0007091220380912303909124030E949935EB
:1040C0009B01AC012F5F310941095109A7E1B0E023
:1040D0000E947634CC24C394DD24DA94ED2CFD2C9C
:1040E000A70196010E945734422F2EE061E370E051
:1040F00088E690E00E94B012C093E007D093DF07FB
:1041000082E090E09093DC078093DB0707E310E008
:104110001093DE070093DD0740E0C501B4010E9463
:10412000E41E88EF0E945A1885E592E10E943F182C
:1041300089E690E09093DC078093DB071093DE071D
:104140000093DD0760912103709122038091230386
:10415000909124030E9499359B01AC012F5F310996
:1041600041095109A4E6B0E00E947634A701960106
:104170000E945734CA01B9010E94BA1E83E592E138
:104180000E943F18D093E007C093DF07DF91CF91E3
:104190001F910F91FF90EF90DF90CF90BF90AF9065
:1041A0009F908F907F906F905F904F9008950E94A6
:1041B000F7371F93CF93DF93EC01162F0E94413402
:1041C000181739F0612FCE01DF91CF911F910C9418
:1041D0004934DF91CF911F910895AF92BF92CF9252
:1041E000DF92EF92FF920F931F93CF93DF93609133
:1041F000530182E090E00E94D9206091520183E057
:1042000090E00E94D9206091510184E090E00E94EA
:10421000D9206091500185E090E00E94D920609102
:104220004F0186E090E00E94D9206091570187E01D
:1042300090E00E94D9206091560188E090E00E94B1
:10424000D9206091550189E090E00E94D9206091C9
:104250008B018AE090E00E94D920609154018BE0AC
:1042600090E00E94D920609159018CE090E00E947A
:10427000D920609120038DE090E00E94D9206091C8
:104280004E018EE090E00E94D92060915A018FE0AB
:1042900090E00E94D9206091FF0280E190E00E94AE
:1042A000D92060911D0381E190E00E94D9206091A6
:1042B000010382E190E00E94D9206091000383E134
:1042C00090E00E94D92084E1E82EF12C10E006E075
:1042D00080914E011817B8F5109F60011124D0E0AD
:1042E000C0E0FE01EC0DFD1DE55AFE4F6081C701E7
:1042F0008C0F9D1F0E94D9202196C630D10589F7C9
:10430000670186E0C80ED11C88E0189FE0011124E7
:10431000C25FDE4F8EE0E80EF11C69812296C60175
:104320000E94D920560182E0A80EB11CFE013297EE
:104330006081C60101960E94D9206501AE14BF04B8
:1043400061F71F5FC5CFDF91CF911F910F91FF9054
:10435000EF90DF90CF90BF90AF9008958F929F9293
:10436000AF92BF92CF92DF92EF92FF92CF936FEF17
:1043700070E089E00E94CF158BEA94E00197F1F795
:104380008EE00E94DD187C018AE00E943C1590912D
:10439000CE02981729F091E0909318038093CE02F3
:1043A000809101019FEF980F90930101811106C048
:1043B0000E940B1990931F0380931E0360912103A9
:1043C0007091220380912303909124030E949935D8
:1043D00089E00E94CF158090FB029090FC02A09093
:1043E000FD02B090FE02B70190E080E00E9422330F
:1043F000A50194010E94BA342DEC3CEC4CE45DE341
:104400000E948333A50194010E94BB346093FB0298
:104410007093FC028093FD029093FE020E94E31CC5
:10442000609128037091290390E080E00E9422337C
:104430006B017C012091D5023091D6024091D702C8
:104440005091D8020E941D338111BAC020911403EB
:10445000309115034091160350911703C701B6011F
:104460000E94BA346B017C0120E030E0A9010E9477
:10447000CF3518160CF09AC020E030E040EA50E446
:10448000C701B6010E94CF3518160CF499C060918F
:1044900012037091130390E080E00E942233209178
:1044A00014033091150340911603509117030E9495
:1044B000BA346B017C0120E030E0A9010E94CF35C5
:1044C00018160CF08CC0C701B6010E94A03570937D
:1044D000D4026093D3026530710508F084C08091E6
:1044E0008C01811105C08091580181110E94C2196F
:1044F00081E080938C011092580180912803909163
:104500002903853F21E0920710F0109200012091CD
:104510000001211141C0843F9140F0F56FEF70E040
:1045200089E00E94CF150E94C219C1E0C09300012A
:104530000E94DF1D0E94ED20C09318038EE00E94B0
:10454000DD18BC0190E080E00E9422336093FB0202
:104550007093FC028093FD029093FE0210920C0374
:1045600080911203909113032CE231E030933103D8
:104570002093300320E233E030932F0320932E0367
:104580002AE030E030932D0320932C03880F991FED
:1045900090932B0380932A03CF91FF90EF90DF90AD
:1045A000CF90BF90AF909F908F90089520E030E023
:1045B00040EA50ECC701B6010E941D3387FF67CF68
:1045C0006091140370911503809116039091170365
:1045D0000E94A035709329036093280358CFC70128
:1045E000B601905872CF10928C0187CF0C94413451
:1045F0002F923F924F925F926F927F928F929F92F3
:10460000AF92BF92CF92DF92EF92FF920F931F93E0
:10461000CF93DF938C0186E08093E10781E0809364
:10462000E0071092DF076091EB027091EC02072E19
:10463000000C880B990B0E9424332B013C0145EEA2
:10464000C42E42E0D42E7601C2E0D0E05AE0A52E7E
:10465000B12CBE010D2E000C880B990B0E94243347
:104660009B01AC0160E070E080E291E40E94D435EF
:104670009B01AC01C301B2010E9427350E9499350C
:10468000CB01B5010E94C937F701819391937F0156
:104690002197F8F61093EC020093EB02C9EDD2E0FB
:1046A00094E0E92EF12C22E0822E912C3AE0232E88
:1046B000312CB401092C000C880B990B0E94243377
:1046C0009B01AC0160E070E080E291E40E94D4358F
:1046D0002B013C016091EB027091EC02072E000C63
:1046E000880B990B0E942433A30192010E94273565
:1046F0000E949935CB01B1010E94C937F601208192
:104700003181821B930BF2E3F89FB001F99F700D8A
:104710001124072E000C880B990B0E94243328814A
:1047200039814A815B810E94BB342B013C0120E02E
:1047300030E0A9010E941D3381117CC0488259825A
:104740006A827B8201E022E346E270E060E0C7011A
:1047500004970E94B0128EECA82EBB24BA940FEFDF
:104760001FEF288139814A815B8160E070E080E839
:1047700090E40E94BA342B013C01B5010B2C000CD3
:10478000880B990B0E9424339B01AC01C301B20139
:104790000E94BB340E949935F092DC07E092DB075F
:1047A0007093DE076093DD07F60160817181600F11
:1047B000711F072E000C880B990B0E94BA1E0F5F09
:1047C0001F4FF2E3AF0EB11C0230110551F62496D3
:1047D00021E0821A910882E0C80ED11CECE2EE0EB4
:1047E000F11CF8E8EF16F10409F063CF00E022E0D5
:1047F00040E870E060E090E080E00E94B01220E1CC
:1048000040E860E370E090E080E00E94B012DF9149
:10481000CF911F910F91FF90EF90DF90CF90BF90BD
:10482000AF909F908F907F906F905F904F903F9050
:104830002F900895C301B20190582DEC3CEC4CE44C
:104840005FE30E948333A30192010E94BB3468831B
:1048500079838A839B8376CF4F925F926F927F9208
:104860008F929F92AF92BF92CF92DF92EF92FF9280
:104870000F931F93CF93DF93CDB7DEB72B970FB670
:10488000F894DEBF0FBECDBF90915A01E82FF0E043
:104890009F01220F331F911126C0F901E95CFD4FE2
:1048A00040815181EE24E39400E124E260E370E072
:1048B00080E390E00E94D2122B960FB6F894DEBFF0
:1048C0000FBECDBFDF91CF911F910F91FF90EF9061
:1048D000DF90CF90BF90AF909F908F907F906F9020
:1048E0005F904F900895923009F079C0E356F34EEF
:1048F0004490F901E751FE4FA080B180F12CE12CEA
:1049000004E310E393E0592E27E0622EE414A0F6AE
:10491000F501EE0DFF1D449180E1840F833008F412
:104920005CC081EF7816D1F082EF7816C1F1403F7C
:1049300090F4193710F0085F10E088E0489FA0015C
:104940001124435E5A4E602F70E028E0812F90E0E2
:104950000E948E13185F80EF782E1DC04E39D8F458
:104960001D3710F0085F10E0C02ED12C812E912C45
:10497000459DA00111244D5B5C4E23E0B601C401AE
:104980000E948E1321E042E453E1B601C401039674
:104990000E948E131C5F8FEFE81AF80AB7CF4132DE
:1049A000D0F7193710F0085F10E0C02ED12C812EFF
:1049B000912C469DA0011124455A5D4E27E0B60179
:1049C000C4010E948E1321E042E453E1B601C40108
:1049D00007960E948E13185FDECF742EDCCF80E323
:1049E00090E09093DC078093DB0784E390E0909362
:1049F000DE078093DD0781E08093E107F901EC5346
:104A0000F34E65917491CE0101960E941633CE014A
:104A100001960E948E1D50CFCF93C82F86E00E9432
:104A20003C1521E0892B09F020E0209302030E942D
:104A30007B1380912A0390912B03959587950E9473
:104A4000F8228C2F0E942C240E94AB160E94211960
:104A500086E00E943C15892B51F780910203811159
:104A6000E6CF0E94C2198091EB029091EC02CF91A7
:104A70000895109231031092300328E037E030930C
:104A80002F0320932E0324E630E030932D03209350
:104A90002C03880F991F90932B0380932A0387E0A0
:104AA0000E940C259C01220F331F30933103209369
:104AB0003003865A9F4F880F991F90932F0380933E
:104AC0002E038AE090E090932D0380932C03309383
:104AD0002B0320932A0387E00E940C259C01220FC0
:104AE000331F30933103209330030996880F991FA9
:104AF00090932F0380932E0381E090E090932D03F9
:104B000080932C0330932B0320932A0387E00C948B
:104B10000C252F923F924F925F926F927F928F92CD
:104B20009F92AF92BF92CF92DF92EF92FF920F933C
:104B30001F93CF93DF93182FE0910303F0E0EF561C
:104B4000FE4F80818150990B1092310310923003F7
:104B5000880F991F90932F0380932E0381E090E09C
:104B600090932D0380932C03812F90E0880F991F41
:104B700090932B0380932A0386E00E943C1521E04A
:104B8000892B09F020E0209302031092E00781E0D6
:104B90008093DF0738E3632EE0902A03F0902B0325
:104BA000F594E794AE2C6701DD249601211B3109B1
:104BB000629EC001639E900D1124C80FD91F2097DB
:104BC00009F1662777276C1B7D0B072E000C880BDD
:104BD000990B0E9424332AE939E949E15FE30E94F5
:104BE00083331B012C01BE01DD0F880B990B0E9442
:104BF00024339B01AC01C201B1010E94BB340E946D
:104C00009935EB010E947B138601025011094E0178
:104C100085E0B82E93E0792E7A0CC0900303D12C56
:104C200017FD20C0F601EF56FE4F80818017110658
:104C3000C9F0C4F0E1E9F1E070E060E0CF01815932
:104C400091408C159D0534F48191680F711DF6CF4C
:104C50001E2DA2CF872D8B19680FC401885491098E
:104C60000E943319BA940F5F1F4F88E3880E911C7E
:104C7000B110D3CFE1E9F1E090E080E09F0121594C
:104C800031402C153D0524F42191820F911DF6CF62
:104C90008E0D0E942C240E94AB160E94211986E0E2
:104CA0000E943C15892BA1F6809102038111D0CF7F
:104CB0000E94C2198A2DDF91CF911F910F91FF9011
:104CC000EF90DF90CF90BF90AF909F908F907F90AC
:104CD0006F905F904F903F902F9008951F920F928A
:104CE0000FB60F9211242F933F934F935F936F93BF
:104CF0007F938F939F93AF93BF93EF93FF9382E341
:104D000097E00E948414FF91EF91BF91AF919F9122
:104D10008F917F916F915F914F913F912F910F9064
:104D20000FBE0F901F9018951F920F920FB60F9203
:104D300011242F938F939F93EF93FF93E09142075A
:104D4000F09143078081E0914807F091490782FD87
:104D50001BC0908180914B078F5F8F7320914C0710
:104D6000821741F0E0914B07F0E0EE5CF84F958F31
:104D700080934B07FF91EF919F918F912F910F900F
:104D80000FBE0F901F9018958081F4CF1F920F9245
:104D90000FB60F9211242F933F938F939F93AF934E
:104DA000BF938091EE029091EF02A091F002B0913A
:104DB000F1023091ED0223E0230F2D3758F50196D3
:104DC000A11DB11D2093ED028093EE029093EF029E
:104DD000A093F002B093F1028091F2029091F3025D
:104DE000A091F402B091F5020196A11DB11D80932E
:104DF000F2029093F302A093F402B093F502BF91F4
:104E0000AF919F918F913F912F910F900FBE0F9077
:104E10001F90189526E8230F0296A11DB11DD2CF31
:104E20001F920F920FB60F9211242F933F934F931F
:104E30005F936F937F938F939F93EF93FF9383B1D0
:104E4000817029B19091F802981709F49DC030E063
:104E5000220F232F221F330B922F8093F8024091B1
:104E6000F702241709F490C02093F70220912C0335
:104E700030912D03981719F0319521953109409102
:104E80002A0350912B036091300370913103240F5A
:104E9000351F261737070CF48BC020912C03309157
:104EA0002D03981719F031952195310940912A0366
:104EB00050912B0360912E0370912F03240F351F07
:104EC000621773070CF46FC040912C0350912D03AF
:104ED000981719F051954195510920912A03309165
:104EE0002B03240F351F30932B0320932A0341E01B
:104EF000981340E02091F602421709F440C0209137
:104F00002C0330912D03981719F031952195310913
:104F100060912A0370912B03E0913003F0913103EB
:104F2000260F371F2E173F070CF44CC020912C037F
:104F300030912D03981719F0319521953109609121
:104F40002A0370912B03E0912E03F0912F03260F7B
:104F5000371FE217F3078CF120912C0330912D03BA
:104F6000981719F031952195310980912A03909174
:104F70002B03820F931F90932B0380932A0340935C
:104F8000F60281E080931803FF91EF919F918F913A
:104F90007F916F915F914F913F912F910F900FBE35
:104FA0000F901F90189520912E0330912F039BCFC7
:104FB000209130033091310396CF80912E03909150
:104FC0002F03D9CF8091300390913103D4CF18951E
:104FD000E2E3F7E01382128288EE93E0A0E0B0E013
:104FE00084839583A683B78385EA92E09183808347
:104FF00085EC90E09587848784EC90E0978786879E
:1050000080EC90E0918B808B81EC90E0938B828B95
:1050100082EC90E0958B848B86EC90E0978B868B6E
:10502000118E128E138E148EEFECF7E01382128223
:105030001682178280E1808715821482128687EBA0
:1050400092E091838083158614861786168681E008
:10505000808B118A828B138A0895CF93DF93CDB70B
:10506000DEB72C970FB6F894DEBF0FBECDBF789495
:1050700084B5826084BD84B5816084BD85B582605D
:1050800085BD85B5816085BD80916E00816080930E
:105090006E00109281008091810082608093810077
:1050A0008091810081608093810080918000816087
:1050B000809380008091B10084608093B1008091E2
:1050C000B00081608093B00080917A00846080930A
:1050D0007A0080917A00826080937A0080917A00D1
:1050E000816080937A0080917A00806880937A0052
:1050F0001092C1001092B90088E48093B8000E9419
:10510000A11680E00E94971609E712E2F801849147
:105110000E9497160F5F1F4FF2E208391F07B1F781
:105120000E948F1611E01093B8000E94AB1681E226
:105130008093D70760E08EE00E94931560E08FE0D7
:105140000E949315609121037091220380912303A3
:10515000909124030E94A035062F85E00E949315AC
:10516000602F89E00E94931562E087E00E9493150A
:1051700062E088E00E94931562E086E00E94931549
:1051800062E08AE00E9493156FEF70E089E00E9470
:10519000CF1560E085E00E94651580917A008760F8
:1051A00080937A0080917A00886080937A00789466
:1051B00010936B00109368001BBB90E080E00E948E
:1051C000F622182F81E090E00E94F622912F8F3175
:1051D000984009F0C9C082E090E00E94F622182FA2
:1051E00083E090E00E94F622912F909353018093E8
:1051F000520184E090E00E94F622182F85E090E0B2
:105200000E94F622912F909351018093500186E0E5
:1052100090E00E94F62280934F0187E090E00E9488
:10522000F6228093570188E090E00E94F622809356
:10523000560189E090E00E94F622809355018AE0B1
:1052400090E00E94F62280938B018BE090E00E9418
:10525000F62291E0811101C090E0909354018CE01E
:1052600090E00E94F62291E0811101C090E09093BD
:1052700059018DE090E00E94F622809320038EE099
:1052800090E00E94F622282E80934E018FE090E05D
:105290000E94F62280935A0180E190E00E94F6225B
:1052A00091E0811101C090E09093FF0281E190E0D4
:1052B0000E94F62280931D0382E190E00E94F62274
:1052C000182F83E190E00E94F622912F9093010322
:1052D000809300034EE0842E41E0942E5BE5A52EE2
:1052E00051E0B52E64E1E62EF12C312C231409F4A3
:1052F00047C010E000E0C701800F911F0E94F62216
:10530000F501E00FF11F80830F5F1F4F063011057D
:1053100091F7670136E0C30ED11C4EE0E40EF11C9C
:105320003401C6010E94F622082F10E0102F00273A
:10533000D3010D931C932601B2E04B0E511CC60104
:1053400001960E94F622082BF301019311933F016D
:1053500062014E145F0429F73394F8E08F0E911C1C
:1053600026E0A20EB11CC2CF68E090E080E00E946F
:10537000D9206FE181E090E00E94D9200E94ED20C9
:105380001091FF0280EC111101C088EC0E94C81638
:1053900080EA111101C081EA0E94C8161092190317
:1053A00080E280931A0380E480931B0380E680935D
:1053B0001C038091000390910103892B19F10E9435
:1053C0007B1367E088E290E00E94331987E00E9437
:1053D0002C240E94AB1668EE73E080E090E00E94FF
:1053E00051160E94C2190E94C2190E94C21990E06F
:1053F00080E00E943925209100033091010382173B
:105400009307E9F60E9463189093FA028093F902D9
:105410000E940B1990931F0380931E030091520169
:105420001091530110931303009312038EE00E9416
:10543000DD18BC0190E080E00E9422336093FB0203
:105440007093FC028093FD029093FE020E949F18CD
:105450000E94E31C20E030E040EA51E46091140334
:105460007091150380911603909117030E94BB342D
:105470006B017C01B80190E080E00E9422339B0127
:10548000AC01C701B6010E941D3387FF05C070E063
:1054900060E089E00E94CF1583B181708093F802AB
:1054A00089B190E0880F892F881F990B8093F702AC
:1054B0002091F8029091F70281E0291380E0809317
:1054C000F6028CE291E0909331038093300380E206
:1054D00093E090932F0380932E038AE090E09093C3
:1054E0002D0380932C03000F111F10932B030093A7
:1054F0002A030E94831660930E0370930F03809318
:105500001003909311030E94C2190E94C2192090A7
:105510002A0330902B03A101559547955A87498757
:10552000509313034093120386E00E943C15482ECB
:1055300081118DC080910C03882309F488C00E94DA
:10554000C2190E9483166B017C01C0920803D0929D
:105550000903E0920A03F0920B0386E00E943C15D7
:10556000892B59F40E9483166C197D098E099F09B5
:10557000643F71408105910580F30E9483166C1988
:105580007D098E099F09643F71408105910508F4EA
:105590005AC46FEF70E089E00E94CF150E94C219D3
:1055A000512CAAE06A2E712C10920303852D0E94C3
:1055B0008925582EB9E0B81738F1E82FF0E0ED5101
:1055C000F54D0C94DD37ED2A9A2D142E802E8E2E5B
:1055D000BF2ECD2EEE2EF92E032FF6E0FF2E81E00A
:1055E00080930303852D0E948925582EE2E08E17B3
:1055F00009F439C2E81708F4E9C0882309F413C193
:10560000F1E08F1709F412C10E94ED2081E0809330
:105610001803E985FA85F0931303E09312038CE2F3
:1056200091E0909331038093300380E293E0909374
:105630002F0380932E038AE090E090932D038093B4
:105640002C03C1018E7F90932B0380932A034092F9
:105650000C0380912503882309F110915501112332
:10566000E9F00E948316C0900403D0900503E090F7
:105670000603F09007036C197D098E099F0928EE37
:1056800033E040E050E00E948934211738F0109256
:1056900025030E94C21981E080935801809118036C
:1056A0008823F1F180912603882351F120E030E036
:1056B00040EA51E460911403709115038091160340
:1056C000909117030E94BB346B017C01609112031F
:1056D0007091130390E080E00E9422339B01AC01A3
:1056E000C701B6010E941D3387FF05C070E060E06E
:1056F00089E00E94CF150E94C21981E08093580171
:105700001092180310922603109227030E9483160A
:1057100060930E0370930F03809310039093110313
:105720000E94831600910E0310910F032091100325
:1057300030911103601B710B820B930B20E63AEE44
:1057400040E050E00E948934122F20930D03809195
:10575000260381110BC080915701882339F0281747
:1057600028F081E0809326030E94C21980912703CC
:1057700081110BC080915601882339F0181728F049
:1057800081E0809327030E94C2190E94AE210E94EB
:10579000D01A0E9483168091D807F62FF81B8F2FFE
:1057A0009091D907992309F464C3F093DA07109212
:1057B000D90780E090E0892B09F4A9CE0E947014EB
:1057C000882309F4A4CE0E940000A1CE23E0821712
:1057D00009F44CC134E0831317CF80914E01883017
:1057E00008F0FDCE91E0980F90934E018093200336
:1057F0000E94E019E0912003B8E0EB9FF001112432
:10580000E25FFE4F28ED30E03183208344E351E036
:105810005383428386E891E095838483AEE1B0E0D0
:10582000B783A683DCCE0E94DF1DD9CE8E010F5F29
:105830001F4F612C712C4301639478EEC72E73E0E7
:10584000D72EAA24A394B12CEE24E394E091200354
:1058500044E0E49FF0011124C3010197E80FF91F10
:10586000EE0FFF1FE25FFE4F808191819093130343
:1058700080931203A8ECB0E0B0933103A0933003FF
:10588000D0922F03C0922E03B0922D03A0922C032E
:10589000880F991F90932B0380932A03E09258015D
:1058A00086E00E943C1521E0892B09F020E020933E
:1058B00002030E947B13B2E0B093E1070E94AE2185
:1058C0000E94D01A1092DC071092DB071092DE07BC
:1058D0001092DD078EEB92E20E943F18C401B301E3
:1058E0000E94BA1E8BEC92E00E948E1D80918C016A
:1058F0001092DC071092DB07882309F48CC0E0E1EA
:10590000F0E0F093DE07E093DD0781EB92E20E9486
:105910003F181092DC071092DB0720E230E0309352
:10592000DE072093DD078AEA92E20E943F18609129
:105930002A0370912B0375956795072E000C880B31
:10594000990B0E94BA1E0E9421190E94AB1686E094
:105950000E943C15892B09F0ACCF80910203811184
:10596000A8CF80912A0390912B0395958795D80114
:105970008D939D938D010E94C2196AE070E080E0D2
:1059800090E00E945116BFEF6B1A7B0A8B0A9B0AAC
:10599000E4E06E1671048104910409F057CF6FEFB3
:1059A00070E089E00E94CF158BEA94E00197F1F74F
:1059B0000E949F180E94A0353B0178876F83A980C1
:1059C000BA800B811C81C5014E968017910708F0A3
:1059D00006CECD80DE80C8014E968C159D0508F060
:1059E000FECD87E08093030380E00E948925882311
:1059F00009F4F5CDE091200328E0E29FF0011124A5
:105A0000E25FFE4FB182A08213830283D582C482FB
:105A100077826682E4CD40E150E05093DE07409308
:105A2000DD0784EA92E20E943F186091FB027091C8
:105A3000FC028091FD029091FE020E94A03590E050
:105A400080E04AE00E949B1D1092DC071092DB0769
:105A500080E290E09093DE078093DD0788E992E290
:105A60000E943F1870CF0E94E019B9CD87E0809363
:105A7000030380914E01813009F4B1CD80E00E9492
:105A80008925882309F4ABCD8091200390914E01A4
:105A9000492F4150550B9A018417150639F481504E
:105AA00080932003915090934E0199CDE82FF0E020
:105AB000E217F307BCF78F9D8001112450E040E00E
:105AC0006F016FEFC61AD60AB801640F751F655AC9
:105AD0007E4FDB011696EC901697EC924F5F5F4F6E
:105AE0004630510589F7D60113E0AA0FBB1F1A955E
:105AF000E1F7A25FBE4F4D915C91119703E0EE0F6D
:105B0000FF1F0A95E1F7E25FFE4F51834083129633
:105B10004D915C9113975383428314964D915C9100
:105B200015975583448316964D915C915783468310
:105B30008F5FBCCF82E08093030310E0E8E2CE2EBB
:105B4000D12CFCE2AF2EBB24B394A0E28A2EA3E0BA
:105B50009A2EB4E1EB2EF12C812F0E948925182F6B
:105B6000813029F130F0823009F441C00E94ED20EB
:105B70001BCD8091520190915301B0923103A092BC
:105B8000300390922F0380922E0370922D03609227
:105B90002C03880F991F90932B0380932A0381E194
:105BA0000E940C259093530180935201D5CF809190
:105BB000500190915101D0923103C0923003E0E93D
:105BC000F1E0F0932F03E0932E0370922D03609287
:105BD0002C03880F991F90932B0380932A0382E153
:105BE0000E940C259093510180935001B5CF809174
:105BF0004F0190E0F0923103E092300328EC30E066
:105C000030932F0320932E0370922D0360922C0368
:105C1000880F991F90932B0380932A0383E10E949E
:105C20000C2580934F0198CF83E080930303F12CE0
:105C300001E010E08F2D0E948925F82E31E08317B6
:105C400009F43FC0831700F142E084138FCF8091A5
:105C5000550190E0109231031092300348E651E074
:105C600050932F0340932E0370922D0360922C03C8
:105C7000880F991F90932B0380932A0387E10E943A
:105C80000C2580935501D6CF8091570190E010925A
:105C9000310310923003ACE3B0E0B0932F03A09334
:105CA0002E0310932D0300932C03880F991F9093BC
:105CB0002B0380932A0385E10E940C2580935701D2
:105CC000B9CF8091560190E01092310310923003C9
:105CD000E8E7F0E0F0932F03E0932E0325E030E0B7
:105CE00030932D0320932C03880F991F90932B033F
:105CF00080932A0386E10E940C25809356019ACF57
:105D000084E080930303809154010E94892591E0EF
:105D1000811101C090E09093540146CC10E0B9E0AD
:105D2000EB2E05E0D02EE0920303812F0E948925FF
:105D3000182F882321F08130E1F000E009C0D092D3
:105D4000030380918B010E94892580938B0101E0E0
:105D5000F090FF0280ECF11001C088EC0E94C816A0
:105D600080EAF11001C081EA0E94C8160111DBCF60
:105D7000FDCE8091FF0281278093FF02E8CF86E06D
:105D800080930303809159010E94892591E081113C
:105D900001C090E09093590107CC80911D0390E0E1
:105DA0001092310310923003A4EFB1E0B0932F03AF
:105DB000A0932E0321E030E030932D0320932C0399
:105DC000880F991F90932B0380932A0386E00E94EB
:105DD0000C2580931D030E94C219E6CB809100031D
:105DE000909101030E943925909301038093000351
:105DF000F2CF88E08093030380915A010E948925A5
:105E000080935A01D1CB0E947B13EE24E39400E3EC
:105E100020E345EC52E270E060E088E290E00E940E
:105E2000D2120E94AB1664E670E080E090E00E941F
:105E3000511686E00E943C15892BD9F78091020308
:105E40008111F7CFC8CF8091250391E089278093F6
:105E50002503882351F00E948316609304037093F6
:105E60000503809306039093070381E08093180352
:105E7000EECB9091D707F91748F48F5F891708F098
:105E800098CC81E083BF889513BE93CC81E080934A
:105E9000D9076093D8078091D3079091D4070196D2
:105EA0009093D4078093D307A0902803B090290340
:105EB00025EFA21621E0B20608F029C18091270340
:105EC000882309F402C16FEF70E089E00E94CF15CA
:105ED0000E947B1309E113E07DE1272E73E0372E4A
:105EE000E2E08E2E912CA12CB12CF3E04F2E512C00
:105EF000612C712C0E94BE32A50194010E9457347E
:105F0000AB01BC014150510961097109D8018C9163
:105F1000682F640F613808F04EC06C9319860E9498
:105F2000BE32F985CF2ED12CF12CE12CA3019201A8
:105F30000E9457346D5F7F4F8F4F9F4FA70196018F
:105F40002617370748075907D4F5D801EC90F12CEC
:105F50000E94BE3224E130E040E050E00E9457341D
:105F60006A507109810991096E0D7F1D60347105B8
:105F700030F421E040E890E080E00E94D516F8017E
:105F8000E080F12C0E94BE3224E130E040E050E09D
:105F90000E945734DC01CB010A97A109B1098E0D8B
:105FA0009F1D21E040E470E060E00E948712F985C7
:105FB000FF5FF987B4CF6058F8016083AFCF0F5F00
:105FC0001F4F2016310609F095CF0E9483160E94BC
:105FD000223320E030E04AE755E40E9427350E9452
:105FE00024366B017C0120E030E040E853E40E945D
:105FF000833320E030E040E853E40E94BB342B01BF
:106000003C0110E000E0B801012E000C880B990B58
:106010000E942433A30192010E941D3387FF25C0F3
:106020000E94BE324B015C010E94BE3269877A87B2
:106030008B879C87C501B40120E430E040E050E04C
:106040000E9457344B0169857A858B859C8520E8B1
:1060500030E040E050E00E945734CB0141E0B40111
:106060000E9469120F5F1F4FCECF80915901882384
:1060700049F10E94BE3220E130E040E050E00E9451
:10608000573468507109810991090E9424334B01EA
:106090005C0120E030E040E852E4C701B6010E9414
:1060A000833320E030E040E852E40E94BB349B019F
:1060B000AC01C501B4010E94BB340E94993585E052
:1060C0000E94CF150E94AB1674CB8091260312E07C
:1060D00081111EC08091250313E0811119C08091A8
:1060E0008C0114E0811114C020E030E044E353E45B
:1060F00060912103709122038091230390912403E6
:106100000E941D3315E087FD03C016E001C010E0BA
:1061100080918B01882309F481C10E947B1301E0E7
:1061200020E440E870E060E090E080E00E94B0127F
:1061300081E08093E1078093E0071092DF07E12C74
:1061400000E120E143E554E270E060E090E080E0AF
:106150000E94D21283E190E09093DC078093DB07EA
:1061600084E090E09093DE078093DD078091200328
:1061700026E0829FC0011124855A9E4F0E948E1DE9
:1061800085E390E09093DC078093DB0781E090E06B
:106190009093DE078093DD0782E08093E107C12EB4
:1061A000D12C80915A01CC0CDD1C8111EAC0F60182
:1061B000ED56FD4F408151810EE02CE161E070E031
:1061C00080E590E00E94D212F601EB57FD4F40812E
:1061D0005181E12C0EE02EE061E070E081E790E07B
:1061E0000E94D21281E08093E1070E949F1820E074
:1061F00030E040EA52E40E94CF3518160CF4E0C0BB
:10620000E12C0EE02EE041E154E262E170E082E038
:1062100090E00E94D21260911E0370911F0390E0E3
:1062200080E00E94223320E030E048EC52E40E94FB
:1062300027356B017C0160911D0370E090E080E0E8
:106240000E9424339B01AC01C701B6010E941D339B
:1062500087FDCAC0E12C0EE02EE045EF53E262E27A
:1062600070E082E090E00E94D21203E110E010930F
:10627000DC070093DB0740E150E05093DE074093DA
:10628000DD070E949F1841E00E94E41E88EF0E94F3
:106290005A1883EF93E20E943F181093DC07009393
:1062A000DB0788E190E09093DE078093DD070E9492
:1062B0006318BC0190E080E00E94223320E030E0CF
:1062C0004AE754E40E94273542E00E94E41E81EF31
:1062D00093E20E943F181093DC070093DB0780E2F3
:1062E00090E09093DE078093DD0760911E0370912C
:1062F0001F0390E080E00E94223320E030E04AE774
:1063000054E40E94273541E00E94E41E8FEE93E2A0
:106310000E943F181093DC070093DB0788E290E0AF
:106320009093DE078093DD0789EE93E20E943F1889
:1063300089E390E09093DC078093DB0782E190E0B3
:106340009093DE078093DD0784E08093E1076091FE
:10635000280370912903653F91E0790708F458C03C
:1063600085EE93E20E943F1800E020E248E460E1FD
:1063700070E087E390E00E940C1780E00E94BC1F51
:10638000A1CE83E494E21330C1F058F48FE494E298
:10639000113099F089E494E2123079F08DE294E2C0
:1063A0000CC088E394E2153041F08DE394E215309F
:1063B00020F083E394E2163089F70E943F1804CF5F
:1063C0000E94831652E0660F771F881F991F5A9507
:1063D000D1F728EE33E040E050E00E94893420FFFE
:1063E0000FCF0E94C21917CF0E94831642E0660F9A
:1063F000771F881F991F4A95D1F728EE33E040E0B8
:1064000050E00E94893420FF25CF0E94C2192DCF71
:1064100090E080E04AE00E949B1DA6CF0E947B1383
:106420000E949F1820E030E040EA52E40E94CF35FD
:10643000181694F40E94831632E0660F771F881FA7
:10644000991F3A95D1F728EE33E040E050E00E94E2
:10645000893420FD0E94C21960911E0370911F03B0
:1064600090E080E00E94223320E030E048EC52E4EB
:106470000E9427356B017C0160911D0370E090E064
:1064800080E00E9424339B01AC01C701B6010E9449
:106490001D3387FF12C00E94831622E0660F771F0C
:1064A000881F991F2A95D1F728EE33E040E050E08D
:1064B0000E94893420FD0E94C21987EE93E0A5EF67
:1064C000AA16A1E0BA0608F4C5010E94F82200E06D
:1064D00023E040E860E370E090E080E00E94B012CA
:1064E00081E04CCF8F929F92AF92BF92CF92DF927A
:1064F000EF92FF92CF93DF93EC01688179818A81DB
:106500009B81611571058105910521F464E279EDA6
:106510008BE597E02DE133EF41E050E00E945734E6
:1065200049015A019B01AC01A7EAB1E40E9476340B
:106530006B017C01ACEEB4EFA50194010E948434A0
:10654000C60ED71EE81EF91EF7FE06C081E0C81A67
:10655000D108E10880E8F80AC882D982EA82FB8281
:10656000C701B6019F77DF91CF91FF90EF90DF9049
:10657000CF90BF90AF909F908F9008958F929F92F1
:10658000AF92BF92CF92DF92EF92FF9260918D0116
:1065900070918E0180918F0190919001611571052C
:1065A0008105910521F464E279ED8BE597E02DE119
:1065B00033EF41E050E00E94573449015A019B01FA
:1065C000AC01A7EAB1E40E9476346B017C01ACEE29
:1065D000B4EFA50194010E948434C60ED71EE81EB4
:1065E000F91EF7FE06C081E0C81AD108E10880E86C
:1065F000F80AC0928D01D0928E01E0928F01F09244
:106600009001C701B6019F77FF90EF90DF90CF9088
:10661000BF90AF909F908F90089560938D0170937D
:106620008E0180938F01909390010895FB01DC010E
:1066300005900D920020E1F708950E945F3308F461
:1066400081E00895E89409C097FB3EF49095809509
:10665000709561957F4F8F4F9F4F9923A9F0F92F28
:1066600096E9BB279395F695879577956795B795A6
:10667000F111F8CFFAF4BB0F11F460FF1BC06F5F8C
:106680007F4F8F4F9F4F16C0882311F096E911C09E
:10669000772321F09EE8872F762F05C0662371F0BF
:1066A00096E8862F70E060E02AF09A95660F771FD3
:1066B000881FDAF7880F9695879597F90895990FAF
:1066C0000008550FAA0BE0E8FEEF16161706E807BC
:1066D000F907C0F012161306E407F50798F0621BDD
:1066E000730B840B950B39F40A2661F0232B242BB2
:1066F000252B21F408950A2609F4A140A6958FEFD1
:10670000811D811D08950E9496330C9407340E94C8
:10671000F93338F00E94003420F0952311F00C94E6
:10672000F0330C94F63311240C943B340E9418344B
:1067300070F3959FC1F3950F50E0551F629FF001D4
:10674000729FBB27F00DB11D639FAA27F00DB11DED
:10675000AA1F649F6627B00DA11D661F829F222776
:10676000B00DA11D621F739FB00DA11D621F839FFD
:10677000A00D611D221F749F3327A00D611D231FD3
:10678000849F600D211D822F762F6A2F11249F5721
:1067900050409AF0F1F088234AF0EE0FFF1FBB1F24
:1067A000661F771F881F91505040A9F79E3F5105E3
:1067B00080F00C94F0330C943B345F3FE4F3983E4C
:1067C000D4F3869577956795B795F795E7959F5F8D
:1067D000C1F7FE2B880F911D9695879597F908951F
:1067E00097F99F6780E870E060E008959FEF80EC84
:1067F000089500240A941616170618060906089527
:1068000000240A9412161306140605060895092E8C
:106810000394000C11F4882352F0BB0F40F4BF2BFB
:1068200011F460FF04C06F5F7F4F8F4F9F4F08953B
:1068300057FD9058440F551F59F05F3F71F0479531
:10684000880F97FB991F61F09F3F79F08795089516
:10685000121613061406551FF2CF4695F1DF08C035
:10686000161617061806991FF1CF86957105610552
:1068700008940895E894BB2766277727CB0197F9FA
:106880000895F999FECF92BD81BDF89A992780B5F8
:106890000895262FF999FECF1FBA92BD81BD20BD64
:1068A0000FB6F894FA9AF99A0FBE01960895052E3C
:1068B00097FB1EF400940E946E3457FD07D00E948F
:1068C000893407FC03D04EF40C946E3450954095F7
:1068D000309521953F4F4F4F5F4F0895909580958C
:1068E000709561957F4F8F4F9F4F08950E94AB34F5
:1068F000A59F900DB49F900DA49F800D911D112414
:106900000895B7FF0C9476340E947634821B930B63
:106910000895A1E21A2EAA1BBB1BFD010DC0AA1FE0
:10692000BB1FEE1FFF1FA217B307E407F50720F0F8
:10693000A21BB30BE40BF50B661F771F881F991F73
:106940001A9469F760957095809590959B01AC01BC
:10695000BD01CF010895A29FB001B39FC001A39FC5
:10696000700D811D1124911DB29F700D811D112488
:10697000911D08955058BB27AA270E94D2340C9429
:1069800007340E94F93338F00E94003420F039F4C3
:106990009F3F19F426F40C94F6330EF4E095E7FBD0
:1069A0000C94F033E92F0E94183458F3BA17620799
:1069B00073078407950720F079F4A6F50C943A3410
:1069C0000EF4E0950B2EBA2FA02D0B01B90190010A
:1069D0000C01CA01A0011124FF27591B99F0593F4E
:1069E00050F4503E68F11A16F040A22F232F342F96
:1069F0004427585FF3CF469537952795A795F040E4
:106A00005395C9F77EF41F16BA0B620B730B840BF8
:106A1000BAF09150A1F0FF0FBB1F661F771F881FB0
:106A2000C2F70EC0BA0F621F731F841F48F4879508
:106A300077956795B795F7959E3F08F0B0CF9395FA
:106A4000880F08F09927EE0F9795879508950E9473
:106A50003B350C9407340E94003458F00E94F933FF
:106A600040F029F45F3F29F00C94F03351110C945D
:106A70003B340C94F6330E94183468F39923B1F335
:106A8000552391F3951B550BBB27AA276217730754
:106A9000840738F09F5F5F4F220F331F441FAA1FE8
:106AA000A9F335D00E2E3AF0E0E832D091505040A4
:106AB000E695001CCAF72BD0FE2F29D0660F771F52
:106AC000881FBB1F261737074807AB07B0E809F038
:106AD000BB0B802DBF01FF2793585F4F3AF09E3FBD
:106AE000510578F00C94F0330C943B345F3FE4F3A1
:106AF000983ED4F3869577956795B795F7959F5F00
:106B0000C9F7880F911D9695879597F90895E1E04B
:106B1000660F771F881FBB1F621773078407BA07AA
:106B200020F0621B730B840BBA0BEE1F88F7E09505
:106B300008950E94A0356894B1110C943B340895D7
:106B40000E94203488F09F5798F0B92F9927B751A9
:106B5000B0F0E1F0660F771F881F991F1AF0BA9501
:106B6000C9F714C0B13091F00E943A34B1E00895F1
:106B70000C943A34672F782F8827B85F39F0B93FE3
:106B8000CCF3869577956795B395D9F73EF49095B4
:106B90008095709561957F4F8F4F9F4F08950E940C
:106BA0005F3308F48FEF0895FA01EE0FFF1F309660
:106BB00021053105A1F16115710561F48038BFE34C
:106BC0009B0749F168949038810561F08038BFEFE8
:106BD0009B0741F099234AF5FF3FE1053105210567
:106BE00019F1E8940894E795D901AA2329F4AB2F69
:106BF000BE2FF85FD0F310C0FF5F70F4A695E0F7EA
:106C0000F73950F019F0FF3A38F49F779F930DD081
:106C10000F9007FC9058089546F00C94F63360E00E
:106C200070E080E89FE308954FE79F775F934F936D
:106C30003F932F930E941B372F913F914F915F916C
:106C40000E9483330C9439369F930E9494360F90A0
:106C500007FCEE5F0C94BD360E945F33880B990BE6
:106C6000089529F416F00C94F0330C943A340C94F3
:106C7000F6330E942034A8F39638A0F707F80F9255
:106C8000E8942BE33AEA48EB5FE70E9499330F92CE
:106C90000F920F924DB75EB70F920E946337E8E6EE
:106CA000F0E00E946B364F915F91EF91FF91E59577
:106CB000EE1FFF1F49F0FE57E0684427EE0F441F08
:106CC000FA95E1F74195550B0E94DD360F9007FECE
:106CD0000C94D1360895DF93CF931F930F93FF92B7
:106CE000EF92DF927B018C01689406C0DA2EEF01EF
:106CF0000E949633FE01E894A59125913591459126
:106D00005591A6F3EF010E94D234FE019701A8012C
:106D1000DA9469F7DF90EF90FF900F911F91CF9178
:106D2000DF9108950C94F6330E942034D8F3E89450
:106D3000E0E0BB279F57F0F02AED3FE049EC06C0AA
:106D4000EE0FBB0F661F771F881F28F0B23A62074D
:106D50007307840728F0B25A620B730B840BE39518
:106D60009A9572F7803830F49A95BB0F661F771F9B
:106D7000881FD2F790480C949937EF93E0FF07C033
:106D8000A2EA2AED3FE049EC5FEB0E94D2340E9478
:106D900007340F90039401FC9058E0E9F0E00C9464
:106DA000A5379B01AC0160E070E080E89FE30C94A4
:106DB00027350C94F0330C9497370E942034D8F385
:106DC0009923C9F3940F511DA3F39150504094F0AF
:106DD00059F0882332F0660F771F881F915050407A
:106DE000C1F79E3F51052CF7880F911D9695879509
:106DF00097F908955F3FACF0983E9CF0BB278695CD
:106E000077956795B79508F4B1609395C1F7BB0F77
:106E100058F711F460FFE8CF6F5F7F4F8F4F9F4FA0
:106E2000E3CF0C943B3416F00C9497370C94F63364
:106E300068940C94F0330E942034A8F39923C1F392
:106E4000AEF3DF93CF931F930F93FF92C92FDD27EC
:106E500088232AF02197660F771F881FDAF720E032
:106E600030E040E85FEB9FE3883920F0803E38F067
:106E700021968F770E94BB34EEEAF0E004C00E94B6
:106E8000BB34EBEDF0E00E946B368B01BE01EC01F0
:106E9000FB2E6F5771097595771F880B990B0E9410
:106EA000243328E132E741E35FE30E949633AF2DBC
:106EB0009801AE01FF900F911F91CF91DF910E9439
:106EC000D2340C940734FA01DC01AA0FBB1F9B01DA
:106ED000AC01BF5728F4222733274427507820C01D
:106EE000B75190F4AB2F0024469537952795011C98
:106EF000A395D2F3002071F0220F331F441FB395E6
:106F0000DAF30ED00C94BA3461307105A0E88A0728
:106F1000B94630F49B01AC01662777278827907823
:106F2000309621F0208331834283538308959F3F1D
:106F300031F0915020F4879577956795B795880F34
:106F4000911D9695879597F908959F938F937F93B9
:106F50006F93FF93EF939B01AC010E948333EF91FA
:106F6000FF910E946B362F913F914F915F910C944E
:106F70008333DB018F939F930E947634BF91AF914F
:106F8000A29F800D911DA39F900DB29F900D112483
:106F9000089597FB072E16F4009407D077FD09D0CB
:106FA0000E94E33707FC05D03EF4909581959F4FF2
:106FB0000895709561957F4F0895EE0FFF1F05901E
:106FC000F491E02D0994AA1BBB1B51E107C0AA1F35
:106FD000BB1FA617B70710F0A61BB70B881F991F7A
:106FE0005A95A9F780959095BC01CD01089581E04F
:106FF00090E0F8940C94FC37F894FFCF01FF3C220A
:107000009CCA705158C9C2D4094FD80034018601B6
:107010001E00000000000000000000000000000052
:107020000000000000000000000000000000000060
:107030000000000000000000000000000000000050
:1070400000000000000000000000013C960040012C
:1070500001280F050101014243312E3500000000D7
:107060000000000000000000000000000000000020
:107070000000000000000000000000000000000010
:10708000000000000000000101010000000B0604E8
:10709000040202020203031804FC03E003C403A871
:1070A000038C037003540338031C030003E402C879
:1070B000021804AC0290027402180458023C0274D4
:1070C00002580220023C0274020402E801CC01B022
:1070D0000194018C03780100035C0140012401A8A4
:1070E0000308017402ED04E804E304DC04D604D2CE
:1070F00004C904C604C304BE04BA04B104A7049FAF
:10710000049C049904960490048D048804850482E8
:10711000047D04780475046F046B04670462045DE5
:10712000045904540450044C04490445043C0437F5
:10713000043404CF0F7F0F2F0FDF0E8F0E3F0EEFA3
:107140000D9F0D4F0DFF0CAF0CCF0F5F0C0F0CBF41
:107150000B6F0B1F0BCF0A7F0A2F0A1F0B7F0ADF53
:10716000092F0A1F0B8F093F09EF089F084F08FFDF
:1071700007AF075F070F07BF066F061F06CF051F84
:107180000BAF1093107310F52357103B101F101BFB
:1071900012E311AB1173113B110311CB100000006E
:1071A00000A61406143314F3146414421456140085
:1071B0000000003D17061460185F186E616E0069CC
:0A71C0006E66006F7666002F330044
:107E0000112484B714BE81FFF0D085E080938100F7
:107E100082E08093C00088E18093C10086E0809377
:107E2000C20080E18093C4008EE0C9D0259A86E02C
:107E300020E33CEF91E0309385002093840096BBD3
:107E4000B09BFECF1D9AA8958150A9F7CC24DD24C4
:107E500088248394B5E0AB2EA1E19A2EF3E0BF2EE7
:107E6000A2D0813461F49FD0082FAFD0023811F036
:107E7000013811F484E001C083E08DD089C08234E0
:107E800011F484E103C0853419F485E0A6D080C0E4
:107E9000853579F488D0E82EFF2485D0082F10E0AE
:107EA000102F00270E291F29000F111F8ED06801E7
:107EB0006FC0863521F484E090D080E0DECF843638
:107EC00009F040C070D06FD0082F6DD080E0C81688
:107ED00080E7D80618F4F601B7BEE895C0E0D1E017
:107EE00062D089930C17E1F7F0E0CF16F0E7DF06D8
:107EF00018F0F601B7BEE89568D007B600FCFDCFD4
:107F0000A601A0E0B1E02C9130E011968C91119780
:107F100090E0982F8827822B932B1296FA010C0160
:107F200087BEE89511244E5F5F4FF1E0A038BF0790
:107F300051F7F601A7BEE89507B600FCFDCF97BE46
:107F4000E89526C08437B1F42ED02DD0F82E2BD052
:107F50003CD0F601EF2C8F010F5F1F4F84911BD097
:107F6000EA94F801C1F70894C11CD11CFA94CF0C13
:107F7000D11C0EC0853739F428D08EE10CD085E9AC
:107F80000AD08FE07ACF813511F488E018D01DD067
:107F900080E101D065CF982F8091C00085FFFCCF94
:107FA0009093C60008958091C00087FFFCCF809118
:107FB000C00084FD01C0A8958091C6000895E0E648
:107FC000F0E098E1908380830895EDDF803219F02E
:107FD00088E0F5DFFFCF84E1DECF1F93182FE3DFCA
:107FE0001150E9F7F2DF1F91089580E0E8DFEE27F6
:047FF000FF270994CA
:027FFE00040479
:00000001FF
